:100000004BC0000042C2000040C200003EC20000DF
:100010003CC200000C94844938C2000036C2000083
:1000200034C2000032C200000C947A490C9470492A
:100030002CC200002AC2000028C2000026C2000014
:1000400024C2000022C2000020C200001EC2000024
:100050001CC200000C94304A18C2000016C20000F6
:1000600014C2000012C2000010C200000EC2000044
:100070000CC200000AC2000008C2000006C2000054
:1000800004C2000002C2000000C20000FEC1000065
:10009000FCC10000FAC1000011241FBECFEFD0E266
:1000A000DEBFCDBF0E9400F0D7C10000076342361B
:1000B000B79BD8A71A39685618AEBAAB558C1D3CF9
:1000C000B7CC5763BD6DEDFD753EF6177231BF00BD
:1000D0000000803F05A84CCDB2D44EB93836A902F5
:1000E0000C50B9918688083CA6AAAA2ABE00000036
:1000F000803F08000000BE922449123EABAAAA2A03
:10010000BECDCCCC4C3E00000080BEABAAAAAA3E1D
:1001100000000000BF000000803F00000000000859
:100120004178D3BB4387D1133D190E3CC3BD4282F6
:10013000AD2B3E68EC8276BED98FE1A93E4C80EFB4
:10014000FFBE01C4FF7F3F0000000000FF004C8A9B
:1001500097509545406BA6D8E4B2282EAE90BF26A6
:10016000B14EE86FD0FBE0709A51862C379845323B
:10017000539D06840D971A8CE61E2E0DB41D401655
:100180009AC591F9F786A142660620AFAE19EE270F
:10019000C2BB0EBAB90AAA95CA45040444C1796A19
:1001A00091EE7D3E2E4C960BA96E5A6A9FF56D0519
:1001B000BB8F808DB4F54FC14AE99E674536394FF4
:1001C00075ADF44CB227A939D78036F7C49C7E6A46
:1001D000605F677992B4DD0E4786CD1A6DC6258AB9
:1001E000F464D953D154DB67F78B22BD5CFEA44D78
:1001F000F9A7590EC57E3BF9BA7D430AD39F6C3BE4
:100200000BDEB2875E3710ECC8A6856546290CF177
:10021000D6BCA38C755E4934200DFAE9D7C7B6A7C2
:10022000988A7C6E6155493D32271D1209FFF6EE12
:10023000E5DDD5CEC6BFB9B2ACA6A09A958F8A85AA
:10024000817C78736F6B6864605D5A56FF59E97DF5
:1002500015B150F39942EE9D4F04BC7632F1B2765F
:100260003B03CC98653405D8AC8259320CE7C4A264
:100270008161432509EDD3B9A089725C46321E0B1A
:10028000F8E6D5C4B4A596887A6D6053473C30260D
:100290001B1108FEF5EDE4DCD4CDC6BFB8B1ABA5AB
:1002A0009F99948F8A85807C77736F6B6763605D9D
:1002B000595653504D4A484543403E3C3A383634EF
:1002C00032302E2D2B2A282725242321201F1E1DC6
:1002D0001C1B1A19181716161514131312111110C6
:1002E0000F0F0E0E0D0D0C0C0B0B0B0A0A09090952
:1002F0000808080807070706060606060505050597
:1003000005040404040404030303030303030302B6
:1003100002020202020202020202010101010101C3
:1003200001010101010101010101010101000000C0
:1003300000000000000000000000000000000000BD
:10034000000000000000000000000000FF0C0B0B8C
:100350000B0A0A090909080808080707070606061C
:100360000606050505050504040404040403030347
:100370000303030303020202020202020202020258
:10038000010101010101010101010101010101015D
:10039000010101000000000000000000000000005A
:1003A000000000000000000000000000000000004D
:1003B000000000000000000000000000000000003D
:1003C000000000000000000000000000000000002D
:1003D000000000000000000000000000000000001D
:1003E000000000000000000000000000000000000D
:1003F00000000000000000000000000000000000FD
:1004000000000000000000000000000000000000EC
:1004100000000000000000000000000000000000DC
:1004200000000000000000000000000000000000CC
:1004300000000000000000000000000000000000BC
:1004400000000000000000000000000011241FBE9A
:10045000CFEFD0E2DEBFCDBF1AE1AAECB9E001C018
:100460001D92A037B107E1F719E0A0E0B1E0E0EBA1
:10047000FDEA00E00BBF02C007900D92AA3CB10755
:10048000D9F70E94694A0C94D656BACD2F923F9262
:100490004F925F926F927F928F929F92AF92BF9294
:1004A000CF92DF92EF92FF920F931F93CF93DF9340
:1004B000CDB7DEB727970FB6F894DEBF0FBECDBF1E
:1004C0008EE392E10E94BB1440906F125090701224
:1004D0002091081320FF19C025FD02C00C94070DC0
:1004E000420124FD13C080915412909155129595AC
:1004F0008795480E591E21FD0BC0C12CD12C7601C9
:1005000022FD10C00FEF1FEF1BC0420121FFF5CFEE
:10051000C0905412D0905512EE24D7FCE094FE2CDB
:1005200022FFF0CF00914E1210914F1216950795B1
:10053000009510958091541290915512080F191F33
:100540008091291390912A13A0E0B0E09058A1095E
:10055000B1091C0180910413882311F40C94030D3C
:1005600080913B1390913C13A0E0B0E09058A1091A
:10057000B109B7FF02C00C94BE0DB595A79597952C
:1005800087959C838B832FB72D83F89486E490E125
:100590000E94883340916A1050916B105A834983AE
:1005A000AA2497FCA094BA2C662457FC6094762C5D
:1005B0008091801290918112A3019201280F391F1E
:1005C000411D511DDA01C901009731E0A307B105B2
:1005D00024F08FEF9FEFA0E0B0E0B7FF02C00C94D3
:1005E000110D0E94940E46EC41BB469A31E035B99C
:1005F00025E428B950EF5BB992EA9EB987E881BB40
:1006000000C000C041BB469A35B928B960ED6BB94E
:100610009EB981BB00C000C041BB469A35B928B91C
:100620005BB99EB981BB4B815C8169817A81AA27C4
:10063000469FB12D5703C001749FB00D811D9A1FB5
:1006400056039A0BB00D811D9A1F1124AA2797FDFE
:10065000A095BA2F880D991DAA1DBB1D209174125B
:1006600030917512820F931FA11DB11D009771E08B
:10067000A707B10524F08FEF9FEFA0E0B0E0B7FF30
:1006800002C00C94160D0E94940E46EC41BB469A93
:1006900031E035B921E428B950EF5BB990EA9EB951
:1006A00087E881BB00C000C041BB469A35B928B974
:1006B00060ED6BB99EB981BB00C000C041BB469ADA
:1006C00035B928B95BB99EB981BB910149815A817D
:1006D000AA27249FB12D3503C001529FB00D811D63
:1006E0009A1F34039A0BB00D811D9A1F1124AA275B
:1006F00097FDA095BA2F8C0D9D1DAE1DBF1D20919D
:100700008C1230918D12820F931FA11DB11D40914B
:10071000BC125091BD1260E070E0481759076A079B
:100720007B0714F00C94BF0BDB01CA010E94940EEE
:1007300046EC41BB469A31E035B921E428B950EF87
:100740005BB992EA9EB987E881BB00C000C041BB9B
:10075000469A35B928B960EE6BB99EB981BB00C025
:1007600000C041BB469A35B928B95BB99EB981BB77
:1007700082E491E10E9488332091661130916711E3
:10078000AA27209FB12D319FC001129FB00D811D5E
:100790009A1F309FB00D811D9A1F1124A0E0B0E078
:1007A0000097A105B10509F4E7C79D5FAF4FBF4FA3
:1007B000009751E0A507B10524F08FEF9FEFA0E06F
:1007C000B0E00E94940E46EC41BB469A31E035B948
:1007D00025E428B950EF5BB990EA9EB987E881BB60
:1007E00000C000C041BB469A35B928B960EB6BB96F
:1007F0009EB981BB00C000C041BB469A35B928B93B
:100800005BB99EB981BB6D816FBF7FB77983F89467
:1008100080E790E10E9488332091941030919510E8
:100820003F832E838091821290918312B301A201A3
:10083000480F591F611D711D4115510531E06307B6
:10084000710524F04FEF5FEF60E070E0DB01CA015B
:1008500077FF02C00C94BD0C0E94940E46EC41BB85
:10086000469A31E035B927E428B950EF5BB992EAEE
:100870009EB987E881BB00C000C041BB469A35B92C
:1008800028B960ED6BB99EB981BB00C000C041BB07
:10089000469A35B928B95BB99EB981BB6B817C8119
:1008A0002E813F81AA27629FB12D7303A001369F3D
:1008B000B00D411D5A1F72035A0BB00D411D5A1F36
:1008C0001124662757FD6095762F480D591D6A1D26
:1008D0007B1D8091761290917712480F591F611DF0
:1008E000711D4115510531E06307710524F04FEF8B
:1008F0005FEF60E070E0DB01CA0177FF02C00C949B
:10090000DE0C0E94940E46EC41BB469A31E035B9AC
:1009100023E428B950EF5BB990EA9EB987E881BB20
:1009200000C000C041BB469A35B928B960ED6BB92B
:100930009EB981BB00C000C041BB469A35B928B9F9
:100940005BB99EB981BBB1012E813F81AA27629F0D
:10095000B12D7303A001369FB00D411D5A1F7203C4
:100960005A0BB00D411D5A1F1124662757FD609583
:10097000762F4C0D5D1D6E1D7F1D80918E12909106
:100980008F12480F591F611D711D8091BE129091E9
:10099000BF12A0E0B0E084179507A607B70734F0B0
:1009A00077FF02C00C94ED0CDB01CA010E94940E8B
:1009B00046EC41BB469A31E035B923E428B950EF03
:1009C0005BB992EA9EB987E881BB00C000C041BB19
:1009D000469A35B928B960EE6BB99EB981BB00C0A3
:1009E00000C041BB469A35B928B95BB99EB981BBF5
:1009F0008CE691E10E948833209190113091911101
:100A0000AA27209FB12D319FC001129FB00D811DDB
:100A10009A1F309FB00D811D9A1F1124A0E0B0E0F5
:100A20000097A105B10509F4A4C69D5FAF4FBF4F64
:100A3000009731E0A307B10524F08FEF9FEFA0E00E
:100A4000B0E00E94940E46EC41BB469A31E035B9C5
:100A500027E428B950EF5BB990EA9EB987E881BBDB
:100A600000C000C041BB469A35B928B960EB6BB9EC
:100A70009EB981BB00C000C041BB469A35B928B9B8
:100A80005BB99EB981BB49814FBF3FB73983F894A9
:100A90008AE990E10E9488334091BE105091BF10C6
:100AA0005F834E838091841290918512B301A201DD
:100AB000480F591F611D711D4115510581E06807DF
:100AC000710524F04FEF5FEF60E070E0DB01CA01D9
:100AD00077FF01C057C70E94940E46EC41BB469A6F
:100AE00031E035B921E428B950EF5BB990EA9EB9FD
:100AF00087E881BB00C000C041BB469A35B928B920
:100B000060EE6BB99EB981BB00C000C041BB469A84
:100B100035B928B95BB99EB981BB2B813C816E8107
:100B20007F81AA27269FB12D3703A001729FB00DA8
:100B3000411D5A1F36035A0BB00D411D5A1F112477
:100B4000662757FD6095762F480D591D6A1D7B1D40
:100B50008091781290917912480F591F611D711D73
:100B60004115510581E06807710524F04FEF5FEFF3
:100B700060E070E0DB01CA0177FD25C70E94940E9A
:100B800046EC41BB469A31E035B925E428B950EF2F
:100B90005BB990EA9EB987E881BB00C000C041BB49
:100BA000469A35B928B960ED6BB99EB981BB00C0D2
:100BB00000C041BB469A35B928B95BB99EB981BB23
:100BC00091016E817F81AA27269FB12D3703A00155
:100BD000729FB00D411D5A1F36035A0BB00D411DB7
:100BE0005A1F1124662757FD6095762F4C0D5D1D09
:100BF0006E1D7F1D8091901290919112480F591F88
:100C0000611D711D8091C0129091C112A0E0B0E0F1
:100C100084179507A607B70724F077FDD8C6DB0130
:100C2000CA010E94940E46EC41BB469A31E035B9A8
:100C300025E428B950EF5BB992EA9EB987E881BBF9
:100C400000C000C041BB469A35B928B960EE6BB907
:100C50009EB981BB00C000C041BB469A35B928B9D6
:100C60005BB99EB981BB80919A1190919B11A09123
:100C70009C11B0919D118B2F9927AA27BB27892BF7
:100C80008A2B8B2B09F0F8C58091BF11823009F4B3
:100C90009BC508F093C5813009F460C680E090E000
:100CA0006091B8117091B9110E9485142091B6110C
:100CB0003091B711280F391F3093BB112093BA110F
:100CC0008091961190919711A0919811B0919911DE
:100CD00040919A1150919B1160919C1170919D11BE
:100CE000840F951FA61FB71F80939A1190939B1195
:100CF000A0939C11B0939D11AA27209FB12D319FE5
:100D0000C001129FB00D811D9A1F309FB00D811D33
:100D10009A1F1124A0E0B0E00097A105B10509F4E5
:100D200025C59D5FAF4FBF4F009771E0A707B10585
:100D300024F08FEF9FEFA0E0B0E0F6D746EC41BB88
:100D4000469A31E035B921E428B950EF5BB992EA0F
:100D50009EB987E881BB00C000C041BB469A35B947
:100D600028B960EB6BB99EB981BB00C000C041BB24
:100D7000469A35B928B95BB99EB981BB39813FBF65
:100D80003FB73983F8948091C8109091C910A09111
:100D9000CA10B091CB108B2F9927AA27BB27892B7C
:100DA0008A2B8B2B09F07CC58091ED10823009F4E1
:100DB00022C508F01AC5813009F4C1C580E090E071
:100DC0006091E6107091E7100E9485144091E41044
:100DD0005091E510480F591F5F834E835093E910DF
:100DE0004093E8108091C4109091C510A091C61056
:100DF000B091C7104091C8105091C9106091CA10AD
:100E00007091CB10840F951FA61FB71F8093C81039
:100E10009093C910A093CA10B093CB108091861202
:100E200090918712B301A201480F591F611D711DD6
:100E30004115510581E06807710524F04FEF5FEF20
:100E400060E070E0DB01CA0177FDACC56DD766ECF0
:100E500061BB469A51E055B943E448B970EF7BB99C
:100E600090EA9EB987E881BB00C000C061BB469A8A
:100E700055B948B9E0EEEBB99EB981BB00C000C0DE
:100E800061BB469A55B948B97BB99EB981BB2B81E4
:100E90003C816E817F81AA27269FB12D3703A00157
:100EA000729FB00D411D5A1F36035A0BB00D411DE4
:100EB0005A1F1124662757FD6095762F480D591D3E
:100EC0006A1D7B1D80917A1290917B12480F591FE9
:100ED000611D711D4115510581E06807710524F000
:100EE0004FEF5FEF60E070E0DB01CA0177FD56C5B0
:100EF0001BD766EC61BB469A51E055B947E448B947
:100F000070EF7BB990EA9EB987E881BB00C000C052
:100F100061BB469A55B948B9E0EDEBB99EB981BBC2
:100F200000C000C061BB469A55B948B97BB99EB9AB
:100F300081BB91016E817F81AA27269FB12D370346
:100F4000A001729FB00D411D5A1F36035A0BB00D00
:100F5000411D5A1F1124662757FD6095762F4C0DB1
:100F60005D1D6E1D7F1D8091921290919312480F0E
:100F7000591F611D711D8091C2129091C312A0E092
:100F8000B0E084179507A607B70724F077FD2CC5B6
:100F9000DB01CA01C9D646EC41BB469A31E035B9FE
:100FA00027E428B950EF5BB992EA9EB987E881BB84
:100FB00000C000C041BB469A35B928B960EE6BB994
:100FC0009EB981BB00C000C041BB469A35B928B963
:100FD0005BB99EB981BB8091C4119091C511A0915C
:100FE000C611B091C7118B2F9927AA27BB27892B30
:100FF0008A2B8B2B09F04AC48091E911823009F4C5
:101000002AC408F022C4813009F454C480E090E07E
:101010006091E2117091E3110E9485142091E0111A
:101020003091E111280F391F3093E5112093E4111D
:101030008091C0119091C111A091C211B091C311C2
:101040004091C4115091C5116091C6117091C711A2
:10105000840F951FA61FB71F8093C4119093C511CD
:10106000A093C611B093C711AA27209FB12D319F1D
:10107000C001129FB00D811D9A1F309FB00D811DC0
:101080009A1F1124A0E0B0E00097A105B10509F472
:101090006AC39D5FAF4FBF4F009771E0A707B105CF
:1010A00024F08FEF9FEFA0E0B0E03ED646EC41BBCE
:1010B000469A31E035B923E428B950EF5BB992EA9A
:1010C0009EB987E881BB00C000C041BB469A35B9D4
:1010D00028B960EB6BB99EB981BB00C000C041BBB1
:1010E000469A35B928B95BB99EB981BB39813FBFF2
:1010F0002FB72983F8948091F2109091F310A0916A
:10110000F410B091F5108B2F9927AA27BB27892BB4
:101110008A2B8B2B09F0B5C380911711823009F40B
:1011200081C308F079C3813009F4D3C380E090E033
:1011300060911011709111110E94851440910E114F
:1011400050910F11480F591F5F834E835093131115
:10115000409312118091EE109091EF10A091F01039
:10116000B091F1104091F2105091F3106091F41091
:101170007091F510840F951FA61FB71F8093F21072
:101180009093F310A093F410B093F510809188120F
:1011900090918912B301A201480F591F611D711D61
:1011A0004115510581E06807710524F04FEF5FEFAD
:1011B00060E070E0DB01CA0177FDF8C3B5D566ECED
:1011C00061BB469A51E055B945E448B970EF7BB927
:1011D00090EA9EB987E881BB00C000C061BB469A17
:1011E00055B948B9E0EEEBB99EB981BB00C000C06B
:1011F00061BB469A55B948B97BB99EB981BB2B8171
:101200003C816E817F81AA27269FB12D3703A001E3
:10121000729FB00D411D5A1F36035A0BB00D411D70
:101220005A1F1124662757FD6095762F480D591DCA
:101230006A1D7B1D80917C1290917D12480F591F71
:10124000611D711D4115510581E06807710524F08C
:101250004FEF5FEF60E070E0DB01CA0177FDAAC3EA
:1012600063D566EC61BB469A51E055B941E448B993
:1012700070EF7BB992EA9EB987E881BB00C000C0DD
:1012800061BB469A55B948B9E0EDEBB99EB981BB4F
:1012900000C000C061BB469A55B948B97BB99EB938
:1012A00081BB91016E817F81AA27269FB12D3703D3
:1012B000A001729FB00D411D5A1F36035A0BB00D8D
:1012C000411D5A1F1124662757FD6095762F4C0D3E
:1012D0005D1D6E1D7F1D8091941290919512480F97
:1012E000591F611D711D8091C4129091C512A0E01B
:1012F000B0E084179507A607B70724F077FD6AC307
:10130000DB01CA0111D546EC41BB469A31E035B943
:1013100021E428B950EF5BB990EA9EB987E881BB18
:1013200000C000C041BB469A35B928B960EB6BB923
:101330009EB981BB00C000C041BB469A35B928B9EF
:101340005BB99EB981BB8AEE91E10E9488332091FE
:101350000E1230910F12AA27209FB12D319FC0018C
:10136000129FB00D811D9A1F309FB00D811D9A1FD5
:101370001124A0E0B0E00097A105B10509F4F0C187
:101380009D5FAF4FBF4F009771E0A707B10524F0F5
:101390008FEF9FEFA0E0B0E0C7D446EC41BB469A88
:1013A00031E035B925E428B950EF5BB992EA9EB92E
:1013B00087E881BB00C000C041BB469A35B928B957
:1013C00060EB6BB99EB981BB00C000C041BB469ABF
:1013D00035B928B95BB99EB981BB29812FBF3FB709
:1013E0003D83F89488E191E10E94883340913C115B
:1013F00050913D115A83498380918A1290918B12AA
:10140000480E591E611C711C4114510451E06506BF
:1014100071042CF044244A94542C612C712CD30177
:10142000C20177FCB3C280D446EC41BB469A31E09E
:1014300035B927E428B950EF5BB990EA9EB987E83F
:1014400081BB00C000C041BB469A35B928B960EEE7
:101450006BB99EB981BB00C000C041BB469A35B98B
:1014600028B95BB99EB981BB6B817C8129813A81A6
:10147000AA27629FB12D7303A001369FB00D411DB5
:101480005A1F72035A0BB00D411D5A1F11246627B3
:1014900057FD6095762F480D591D6A1D7B1D809163
:1014A0007E1290917F12480F591F611D711D4115C9
:1014B000510531E06307710524F04FEF5FEF60E005
:1014C00070E0DB01CA0177FD65C22ED446EC41BB5A
:1014D000469A31E035B923E428B950EF5BB992EA76
:1014E0009EB987E881BB00C000C041BB469A35B9B0
:1014F00028B960ED6BB99EB981BB00C000C041BB8B
:10150000469A35B928B95BB99EB981BBB101298129
:101510003A81AA27629FB12D7303A001369FB00DB7
:10152000411D5A1F72035A0BB00D411D5A1F112441
:10153000662757FD6095762F4C0D5D1D6E1D7F1D36
:101540008091961290919712480F591F611D711D3D
:101550008091C6129091C712A0E0B0E08417950761
:10156000A607B70724F077FD3CC2DB01CA01DCD334
:1015700046EC41BB469A31E035B923E428B950EF37
:101580005BB990EA9EB987E881BB00C000C041BB4F
:10159000469A35B928B960EB6BB99EB981BB00C0DA
:1015A00000C041BB469A35B928B95BB99EB981BB29
:1015B0008091181290911912A0911A12B0911B12D9
:1015C0008B2F9927AA27BB27892B8A2B8B2B09F0D6
:1015D00062C180913D12823009F4DFC008F0D7C0AB
:1015E000813009F49BC180E090E0609136127091E7
:1015F00037120E9485142091341230913512280F31
:10160000391F30933912209338124091141250919F
:1016100015126091161270911712C0901812D09086
:101620001912E0901A12F0901B124C0D5D1D6E1DE8
:101630007F1D409318125093191260931A127093E1
:101640001B12AA27209FB12D319FC001129FB00D00
:10165000811D9A1F309FB00D811D9A1F1124A0E09B
:10166000B0E00097A105B10509F477C09D5FAF4FC9
:10167000BF4F009731E0A307B10524F08FEF9FEF34
:10168000A0E0B0E051D346EC41BB469A31E035B919
:1016900027E428B950EF5BB992EA9EB987E881BB8D
:1016A00000C000C041BB469A35B928B960EB6BB9A0
:1016B0009EB981BB00C000C041BB469A35B928B96C
:1016C0005BB99EB981BB3D813FBF2091CA09922F72
:1016D0009C7111E009F010E0922F9370923009F4A0
:1016E000AAC1933009F43EC2913009F4AFC111117F
:1016F00050C280E00E94DF4180918F0D9091900D4B
:10170000A091910DB091920D0196A11DB11D8093F4
:101710008F0D9093900DA093910DB093920D209109
:10172000CA092F5F2093CA0927960FB6F894DEBF27
:101730000FBECDBFDF91CF911F910F91FF90EF9022
:10174000DF90CF90BF90AF909F908F907F906F90E1
:101750005F904F903F902F90089580E090E092CF5F
:1017600080E090E019CE80E090E09FCC80E090E0B7
:10177000E4CA80E090E065C980E090E022C8B7FD4F
:1017800002C00C94960380E090E00C9496038330A2
:1017900009F4BFC0843009F026CF6091181270910F
:1017A000191280911A1290911B1220913A1240E264
:1017B00051E00E94BC258095909517CF833009F4A5
:1017C00099C0843009F06ACA60919A1170919B1196
:1017D00080919C1190919D112091BC1140E251E0AB
:1017E0000E94BC25809590955BCA833009F45DC04A
:1017F000843009F0E3CA6091C8107091C9108091DB
:10180000CA109091CB102091EA1040E251E00E9462
:10181000BC2580959095D4CA833009F475C0843076
:1018200009F084CC6091F2107091F3108091F41063
:101830009091F510209114112111DDC0BB27A92F23
:10184000982F872F8095909573CC833009F457C0DB
:10185000843009F0DBCB6091C4117091C511809187
:10186000C6119091C7112091E61140E251E00E940B
:10187000BC2580959095CCCB86E991E10E944333BD
:1018800003CA8EEE90E10E94433346CC80EC91E196
:101890000E944333B1CB84E192E10E94433399CE5D
:1018A00084EC90E10E9443337FCA8091D8109091DC
:1018B000D91086CA6091C4117091C5118091C6116A
:1018C0009091C7112091E61140E253E00E94BC259F
:1018D0009FCB6091F2107091F3108091F410909171
:1018E000F5102091141121118AC0BB27A92F982F20
:1018F000872F1ECC8091AA119091AB11D1C98091F4
:10190000D4119091D51184CB809102119091031143
:101910000FCC809128129091291267CE60911812F5
:101920007091191280911A1290911B1220913A1203
:1019300021115DC0BB27A92F982F872F56CE60910C
:10194000C8107091C9108091CA109091CB1020914D
:10195000EA1040E253E00E94BC2532CA60919A111D
:1019600070919B1180919C1190919D112091BC11BF
:1019700040E253E00E94BC2593C980E090E0DC0186
:101980000C942C0480E090E0DC01A5C880E090E09D
:10199000DC0149CD80E090E0DC0197CD80E090E073
:1019A000DC01A6CA80E090E0DC0150CA80E090E053
:1019B000DC0104CC80E090E0DC0152CC80E090E0DF
:1019C000DC010C94810480E090E0DC01D7C880E069
:1019D00090E027C980E090E095CC80E090E00C9406
:1019E000D60480E090E0C3CD80E090E0D3CA40E22E
:1019F00053E09CD7FACD40E251E098D723CF40E2A4
:101A000053E094D795CB1C821B820C94C302809028
:101A100054129090551295948794840C951C0C94B4
:101A2000710280E090E0DC010C94F10280E090E033
:101A3000DC010C94430389E592E19DD78091081362
:101A400088700E94CA282091CA096BCE0E94CA39A8
:101A50008091AE14882309F496C08091FB128823EC
:101A600039F081508093FB120E9452198111BAC043
:101A70008091F412882309F47EC02091F2123091F3
:101A8000F31208E912E184E7882E82E1982EACE88F
:101A9000B2E160EB72E190E8A92E92E1B92E44EA3E
:101AA00052E1D12C42C0E81AF90A2E153F0508F47C
:101AB0007901E80EF91EF401F182E082FA01E19069
:101AC000F190AF01F501808191818E159F0508F09D
:101AD00063C0E81AF90A2E153F0508F47901E80EEB
:101AE000F91EF501F182E082FB01E190F190BF0166
:101AF0008D919C9111978E159F0508F05FC0E81A93
:101B0000F90A2E153F0508F47901E80EF91E119621
:101B1000FC92EE92D394F2E08F0E911C129682E02A
:101B2000A80EB11C96E0D91631F1F801E190F190C0
:101B30008F01F401808191818E159F0508F4B3CF48
:101B4000E816F90608F0BACFFC01EE19FF097F018B
:101B50002E173F0708F479018E199F09F40191832C
:101B60008083ACCF22FDDDCD812F0E94242A812FDE
:101B700046D2111135C02091CA09D3CD0196A11DBD
:101B8000B11D0C94BD028091FB12882309F46CCF27
:101B900068CF0E94FF33ADCDE816F90608F0A4CF58
:101BA000FC01EE19FF097F012E173F0708F47901A8
:101BB0008E199F09F5019183808396CFE816F90667
:101BC00008F0A8CFFC01EE19FF097F012E173F078F
:101BD00008F479018E199F0911969C938E939ACFE0
:101BE000AFD5C9CF8091EE0B811103C08091760CE7
:101BF00081110E942D3B8091870D882309F438CFF5
:101C00000E94643A35CFE2E8F8E180818F5F8083FB
:101C1000089555E05A95F1F7000036EC31BB469A2D
:101C200080EE87B997E09AB98DB915B880E488B984
:101C30001BB880E28EB987E481BB82E08A95F1F718
:101C400000C026B199B18CB131BB479A37EE37B994
:101C500037EF3AB932EE3DB9422F4695437050E81E
:101C6000259F90011124422B292F2071422B292FCF
:101C7000269526952870422B96959076492B90E0D4
:101C8000880F991F84709927842B089536EC20EED5
:101C900097E0A0E8F7E4E7EE77EF62EE5FB7F8943D
:101CA00031BB469A27B99AB92DB915B8A8B99BB9CD
:101CB0001EB8F1BB42E04A95F1F700C046B1B9B198
:101CC000BCB131BB479AE7B97AB96DB95FBF55E08E
:101CD0005A95F1F7000042FFE1CF5FB7F89496EC18
:101CE00091BB469A382F330F982F9695232F267045
:101CF0002068482F441F4427441F242B8071836091
:101D0000432F440F4072842B307C832B927090625F
:101D100015B828B98BB99EB987E881BB85E08A954B
:101D2000F1F700005FBF08959C01232F332726950C
:101D30002695722F66EC61BB469A522F550F452FA0
:101D400046704068207133272260352F330F307280
:101D5000322B507C352B272F26952270206215B808
:101D600048B93BB92EB957E851BB969587959695DA
:101D70008795282F61BB469A482F440F382F3695F8
:101D8000221F2227221F642F6670262B2068807155
:101D900099278260942F990F9072982B407C942BF6
:101DA000327015B828B99BB93EB951BB08952F922E
:101DB0003F924F925F926F927F928F929F92AF92DB
:101DC000BF92CF92DF92EF92FF920F931F93CF9328
:101DD000DF93CDB7DEB728970FB6F894DEBF0FBEFE
:101DE000CDBF8D832FB72E83F894282F2595259569
:101DF0002595259580E290E002C0959587952A95D6
:101E0000E2F79D819F70982B86EC81BB469A492F03
:101E1000440F292F2695392F331F3327331F842F43
:101E20008670382B30649071842F880F8072892BD4
:101E3000407C842B2270206491E095B938B98BB92D
:101E40002EB987E881BB35E03A95F1F700002D8186
:101E5000332727FD30953A832983F901EC5CF94F4C
:101E6000C080D12C80E190E08C199D092FEF3FEFCD
:101E7000082E02C0369527950A94E2F702C0220F79
:101E8000331F8A95E2F73C832B83E12CF12C00E091
:101E900010E82FEF3FEF96ECA92E40EEB42E57E05E
:101EA000252E3324339460E4462E70E2572EE7E467
:101EB0006E2EF7EE7F2EA7EF8A2EB2EE9B2E0AC073
:101EC000200F311F16950795AFEFEA1AFA0ACE14C4
:101ED000DF042CF1C9012F83388726DF82E08A9541
:101EE000F1F700C0A1BA469AB7B82AB8BDB835B85C
:101EF00048B81BB85EB861BA92E09A95F1F700C095
:101F000086B189B19CB1A1BA479A77B88AB89DB811
:101F10002F81388585FDD4CF201B310BD3CF86ECA4
:101F200081BB469A81E085B987E488B980EF8BB997
:101F300082E48EB987E881BBB5E0BA95F1F700007D
:101F4000EB81FC812E233F23E981FA81EE0FFF1FF5
:101F5000E554F04F31832083232F3327E981FA8121
:101F6000E956F04F848190E0821B930B97FD1DC0D2
:101F7000059704F53E813FBF28960FB6F894DEBF63
:101F80000FBECDBFDF91CF911F910F91FF90EF90CA
:101F9000DF90CF90BF90AF909F908F907F906F9089
:101FA0005F904F903F902F90089591958195910962
:101FB000059704F3248381E090E0A0E0B0E00D8079
:101FC00004C0880F991FAA1FBB1F0A94D2F7409123
:101FD000970F5091980F6091990F70919A0F842BE1
:101FE000952BA62BB72B8093970F9093980FA093C8
:101FF000990FB0939A0F2D812093FC0FBBCFCF93F5
:10200000882339F18091510A8F5F8093510A85317D
:1020100048F081E09091520A9111CDC08093520A0C
:102020001092510AC091550AC11179C050914F0ABE
:102030009091500AE091560AE13009F4DEC008F4AC
:10204000AFC0E23009F4C4C020E0F0E0E55BF54F3A
:102050002487AFB7F89456EC51BB469A41E045B996
:1020600080E488B91BB880E28EB937E831BB00C084
:1020700000C080E190E00090560A02C0880F991FCE
:102080000A94E2F7282F51BB469A782F770F682FD2
:102090006695221F2227221F972F9670292B2064D6
:1020A0008071972F990F9072982B707C972B62708C
:1020B00045B928B99BB96EB931BB00C000C0E091E9
:1020C000560AF0E0E55BF54F848551BB469A582FE0
:1020D000550F982F9695252F26702064682F661F20
:1020E0006627661F262B682F6071852F880F8072E8
:1020F000862B507C852B9270906245B928B98BB99C
:102100009EB931BBAFBF8091560A90E0019663E063
:1021100070E00E94C8518093560ACF910895409173
:10212000530A4F5F4093530AEAE5FAE0019000201A
:10213000E9F7EB55FA402091540A332727FD3095F3
:10214000C90101966E2F772767FD70950E94C851CF
:10215000F901E55BF54F278530E02038310588F13E
:102160005FEFE82FFF27E7FDF095E55BF54F27854B
:1021700030E02038310550F5F901EC5AF94F9081E3
:10218000403108F457CF8093540A1092530A8111BA
:1021900051CF1C160CF04ECFC150C093550A4ACFF8
:1021A00020914B0A8091520A882309F44ECF8091E6
:1021B0004D0A28274ACF80E08093520A1092510A94
:1021C00031CFF901EC5AF94F5081CBCF9FEFD8CFE7
:1021D000292F2F7780914B0A90914C0A90FD20680F
:1021E00080914D0A90914E0A90FF2FCF8091520A14
:1021F000882309F42ACF205828CF252F2F778091C4
:102200004B0A90914C0A91FD206880914D0A909163
:102210004E0A91FF1ACFEACF4FB7F8948091411040
:1022200096EC91BB469A382F330F982F9695232F13
:1022300026702064582F551F5527551F252B582FC2
:102240005071832F880F8072852B307C832B927086
:10225000906631E035B928B98BB99EB987E881BB62
:102260004FBF089596EC91BB469A582F56955695B8
:1022700056958295880F807E462F440F362F3695CF
:10228000242F26702064962F991F9927991F292B98
:102290006071942F990F9072962B407C942B327022
:1022A000832B55B928B99BB98EB987E881BB85E0E6
:1022B0008A95F1F700000895CF93DF93AADCC82F29
:1022C000D0E0A7DC382F20E0C22BD32B60E081E0E8
:1022D000C9DF60E081E0C6DF61E082E0C3DF60E08B
:1022E00082E0C0DFC095D095CE01DF91CF910895F7
:1022F0006095E1E8F8E19081982B6923608386EC92
:1023000081BB469A362F330F962F9695262F221F84
:102310002227221F832F8670282B20646071832F31
:10232000880F8072862B307C832B9270906C31E00A
:1023300035B928B98BB99EB987E881BB85E08A9504
:10234000F1F70000E0E8F8E180818F5F8083089575
:10235000CF92DF92EF92FF920F931F93CF93DF9371
:1023600090E040E452E46FE070E0F6ECE0EEC7E0AD
:10237000DC2EEE24E394D0E4FD2E00E217E4D7EE49
:10238000C7EFB2EE05C0411551056105710571F148
:10239000F1BB469AE7B9DAB8EDB9E5B8F8B81BB8B9
:1023A0000EB911BB22E02A95F1F700C0A6B1C9B061
:1023B000CCB0F1BB479AD7B9CAB9BDB941505109A0
:1023C00061097109A2FB222720F930E082179307E7
:1023D000D1F6452B462B472B49F0DF91CF911F912A
:1023E0000F91FF90EF90DF90CF900895DF91CF9104
:1023F0001F910F91FF90EF90DF90CF9004CCDF9270
:10240000EF92FF920F931F93CF93DF9390E040E4FE
:1024100052E46FE070E0F6ECE0EE17E0D12EEE242F
:10242000E39400E4F02E00E217E4D7EEC7EFB2EE3B
:1024300005C0411551056105710569F1F1BB469A69
:10244000E7B9DAB8EDB9E5B8F8B81BB80EB911BB01
:1024500022E02A95F1F700C0A6B1A9B1ACB1F1BB59
:10246000479AD7B9CAB9BDB9415051096109710933
:10247000A1FB222720F930E082179307D1F6452BE4
:10248000462B472B41F0DF91CF911F910F91FF9089
:10249000EF90DF900895DF91CF911F910F91FF9002
:1024A000EF90DF90B0CBCF93DF93E8E8FDE0808141
:1024B000CAE8DDE0688190E070E00E94C851A09118
:1024C0008B0DB0918C0DA80FB91F2C913FB7F894CC
:1024D000808190E00196688170E00E94C8518083FD
:1024E0003FBF822FDF91CF91D1CB0F931F93072F47
:1024F000069510E00F771127282F2F774091AC1405
:102500004F704069E0918319F091841963E070E0A5
:1025100083E899E109951F910F9108950F93262F54
:102520004F772F778F708068E0918319F09184192D
:10253000042F482F63E070E083E899E109950F913B
:102540000895EF92FF920F931F93CF93DF93EC01C7
:10255000162FF42EE22E8091A819843071F1C2302A
:10256000D10509F453C0C330D10571F1C130D10593
:10257000F9F1C430D105C8F5E0919F19F091A01987
:10258000309739F00E2D2F2D412FBE0183E899E1B0
:102590000995E091A119F091A219309739F00E2D0B
:1025A0002F2D412FBE0183E899E10995DF91CF914D
:1025B0001F910F91FF90EF900895E0919D19F09178
:1025C0009E193097F9F6D8CF862F807F803A09F48C
:1025D0008DC008F041C0803809F456C0803961F6DA
:1025E000E0918719F091881942C0C0E0D0E0C4CFD3
:1025F000683F50F1E0919919F0919A19309709F4D8
:10260000BBCF612F83E899E10995C3CF862F807FE7
:10261000803D09F455C0803F09F440C0803C09F07A
:10262000ABCFE0919119F0919219309709F4A4CFB2
:10263000133F09F43FC0113FE9F1612F6F704F2D37
:1026400083E899E10995A5CF663F09F095CFE09120
:102650009B19F0919C19D2CF803ED9F0803FA9F10F
:10266000803B09F089CFE0918519F0918619309768
:1026700009F482CF123F99F1612F6F702E2D4F2DEB
:1026800083E899E1099585CFE0918919F0918A193C
:10269000EECFE0918D19F0918E19E9CF633F59F19A
:1026A000613F09F069CFE0919719F091981930973F
:1026B00009F462CF4F2D612F83E899E1099569CF25
:1026C000E0919319F0919419B0CF623F09F054CF83
:1026D000E0918F19F0919019309709F44DCF2E2D7C
:1026E0004F2D62EF83E899E1099553CFE0918B1963
:1026F000F0918C19BCCFE0919519F0919619309713
:10270000C9F63ACF21E02093550A0097A9F010921C
:10271000540ABC018BE59AE00E94DC55EAE5FAE038
:1027200001900020E9F7EB55FA40E65AF54F80E2B8
:1027300090E09183808308958FEF8093540A0895E9
:1027400080918213882319F0815080938213089519
:102750001092970F1092980F1092990F10929A0F53
:102760008FEF8093FC0F809374138FEF9FEFDC014A
:102770008093751390937613A0937713B093781387
:1027800008958F929F92AF92BF92CF92DF92EF9275
:10279000FF920F931F934A015B0168017901BC010D
:1027A00080E090E00E940C539058A50194010E9493
:1027B00047520E94B452A70196010E9490540E9471
:1027C000E052CB011F910F91FF90EF90DF90CF90DF
:1027D000BF90AF909F908F9008950F931F93ECE858
:1027E000FAE090E02191922B2AE0EC39F207D1F740
:1027F00031E0911101C030E0E4EAFBE090E020819B
:10280000922B3C962BE0EC3EF207C9F791110BC0DE
:102810004FEF5FEFBA014093F5125093F6126093B9
:10282000F7127093F812332321F09091D616992362
:10283000D1F03093D616882399F080914913909166
:102840004A1300E010E42CE135E440E050E86BE38B
:1028500076E48095909595DF9093FA128093F91223
:102860001F910F91089540918F0D5091900D60919F
:10287000910D7091920D4093F5125093F612609362
:10288000F7127093F812D5CF0F931F93CF93DF9366
:10289000EC018A899B8900E01FEF2FE737E440E0D5
:1028A00050E26BE476E4809590956BDFAC0160E0DC
:1028B00070E0088C04C0440F551F661F771F0A94F0
:1028C000D2F7488759876A877B87DF91CF911F911D
:1028D0000F910895CF93DF93EC017B8B6A8BD4DF4C
:1028E000A98DBB27A1950CF4B095AA0FBB1F11961B
:1028F000288539854A855B850E9473566C877D875C
:102900008E879F87DF91CF910895AC01AA27469FBC
:10291000B12D579F9001749FB00D211D3A1F569FF6
:10292000B00D211D3A1F1124C9010895A72F8F3F13
:10293000F9F0282F2F5F30E0220F331FE82FF0E04F
:10294000EE0FFF1FE40FF51F60817181FA01E20FA6
:10295000F31F80819181861B970B892F9927A89F50
:102960009001A99F300D1124260F371FC90108952A
:102970002EEF31E0E3CF8F929F92AF92BF92CF9232
:10298000DF92EF92FF92CF93DF93EC01CC80DD805A
:10299000EE80FF808F2D9927AA27BB27892B8A2BB2
:1029A0008B2B09F051C08A8D8C849D84AE84BF84AA
:1029B000833009F470C068F5813009F498C08C89BF
:1029C0009D89C80CD91CEA1CFB1CCC82DD82EE82DE
:1029D000FF82BC01705848895989AA27649FB12D8C
:1029E00075039001569FB00D211D3A1F74033A0BD9
:1029F000B00D211D3A1F11242E8B3F8BDF91CF91FB
:102A0000FF90EF90DF90CF90BF90AF909F908F900E
:102A10000895843009F447C0853009F0D0CFB7015C
:102A2000A601E9E07695679557954795EA95D1F720
:102A3000CA015D8B4C8B298D222309F4C2CF80956E
:102A400090959D8B8C8BBDCFE1E0898DE81BE98F44
:102A5000E11155C0C12CD12C7601CC82DD82EE82F1
:102A6000FF82FF27E1950CF4F095DF01AA0FBB1F51
:102A70001196288539854A855B850E9473564B01DE
:102A80005C016C877D878E879F878A8D81113DC011
:102A9000FD8BEC8B94CF46ED54E1C701B60146DFC8
:102AA0009D8B8C8B8ECF2B8922952F7048815981DD
:102AB0006A817B81972F440F551F661F771F892FCF
:102AC000881F8827881F392F3295369537708327BE
:102AD0008927969589278170482B215058F748837C
:102AE00059836A837B83CA015D8B4C8B6ACF7727BE
:102AF0006F2D5E2D4D2DCA015D8B4C8B62CFCC248A
:102B0000CA94DC2CEC2CF12CA8CF823009F050CFE9
:102B10000E942E567D8B6C8B8A8D8C849D84AE8416
:102B2000BF84CC80DD80EE80FF8042CFEF92FF92A9
:102B30000F931F93CF93DF93F82EEFB6F89484E7AB
:102B4000EDEFF2E1DF011D928A95E9F780E090E870
:102B500090931C1380931B13909322138093211343
:102B60002FEF3FEF309326132093251390932A13D2
:102B700080932913309336132093351330931A130F
:102B800020931913909346138093451390935213F7
:102B90008093511390934C1380934B1385E0809353
:102BA000101381E08093111380930A1380930C1308
:102BB0008093121382E08093131346E050E06FEF8E
:102BC00070E083E593E10E94CA5509E513E1C0E096
:102BD000D0E0BE01882777FD8095982F0E940E5384
:102BE0002BEA3AEA4AEA55E40E9490540E94E052E5
:102BF000F801619371938F012196CC30D10549F78B
:102C0000F11008C0EFBEDF91CF911F910F91FF909F
:102C1000EF90089581E08093FD12EFBEDF91CF9198
:102C20001F910F91FF90EF9008958F929F92AF9216
:102C3000BF92DF92EF92FF920F931F93CF93DF9398
:102C40009C01862E912C8114910409F445C081E0E9
:102C5000881A9108A12CB12CAFEF8A1A9A0AAA0AF5
:102C6000BA0ABA2CA92C982C882480E090E0DC01C8
:102C7000A90160E070E0403E51056105710510F565
:102C80005F5F6F4F7F4F762F652F542F4427F4E9F6
:102C9000EF2EFDE0FF2EE80EF91EC0E0D0E000E0D0
:102CA00010E06BBFFA01D790F701E00FF11FD0825F
:102CB00021968E014F5F5F4F6F4F7F4FC115E1E04F
:102CC000DE0779F72F5F3F4F9F5FAF4FBF4F8815EC
:102CD0009905AA05BB0561F61092960F8091940D97
:102CE0009091950DA091960DB091970D28E93DE03A
:102CF0003093950F2093940F853A9641A146B105E4
:102D0000B9F42091980D89E99DE09093950F8093F7
:102D1000940F2093960F81E0DF91CF911F910F9137
:102D2000FF90EF90DF90BF90AF909F908F900895AD
:102D300080E092E0E4E9FDE0DF019C011D9221507A
:102D40003040E1F780E0E8CFEF92FF920F931F93BE
:102D5000CF93DF93E82EEB01FFB6F89461E065DFD7
:102D6000E4E9FEE040E051E004C0A901211531058D
:102D7000F9F09A012150310992919923B1F39A0106
:102D80008A010F5F1F4FE092E916EAEEF6E184E94F
:102D90009DE0A901BC01CF010E94B05519830883B1
:102DA000FFBEDF91CF911F910F91FF90EF9008959B
:102DB00001E010E020E030E0E6CF1F93CF93DF93F7
:102DC0001FB7F89461E031DF882309F496C080E0F2
:102DD000ADDE109253138FEF8093541380935513ED
:102DE0008093561380935713809358133091960F06
:102DF000332309F47CC0C091940FD091950F20E04B
:102E000089919991E22FF0E0EE0FFF1FE95EFC4EF1
:102E1000918380832F5F293199F7C093940FD093CA
:102E2000950F80E09991DE01D093950FC093940F98
:102E3000E82FF0E0E350FD4E90838F5F873191F7EC
:102E400080910D1380931613323008F450C08D9189
:102E50009D91E22FF0E0EE0FFF1FE95EFC4E9183A3
:102E600080832F5F2E3199F7B093950FA093940F25
:102E7000FD018191F093950FE093940F80931413CB
:102E800011968C911197ED012296D093950FC093D6
:102E9000940F80931513E3E5F3E18991D093950F97
:102EA000C093940F819383E1E935F807B1F78091DE
:102EB000B1149091B2149093521380935113373000
:102EC000B0F0FD013896C9E5D3E1909681919191DA
:102ED00089939993EA17FB07C9F7F093950FE0934D
:102EE000940F1FBF81E0DF91CF911F91089581E082
:102EF0001FBFDF91CF911F91089580E01FBFF9CFD1
:102F0000E4E9FDE080E092E0DF019C011D922150A8
:102F10003040E1F727E02093960F85EA96E1A1E69D
:102F2000B0E080839183A283B383248389E99DE009
:102F30009093950F8093940F0895833061F08931B9
:102F400051F08F3141F091E08F3019F0803109F06C
:102F500090E0892F089591E0892F08958F929F9294
:102F6000AF92BF92EF92FF921F93CF93DF93109295
:102F7000930DC0E0D0E014E26C2F772767FD7095C9
:102F8000872F972F0E940E534B015C012DEB3EE1E2
:102F900040EC55E40E94905420E030E44CE955E4C4
:102FA0000E94DC510E94E0527B0121E33CE043E4BB
:102FB00055E4C501B4010E94905420E030E44CE196
:102FC00056E40E94DC510E94E0521C9FF0011D9FBC
:102FD000F00D1124EA57FC4E86E0E192F192F3865F
:102FE000E286778B668B8150C1F72196C830D10578
:102FF00019F6DF91CF911F91FF90EF90BF90AF90A6
:103000009F908F9008950F931F93CF93DF93E82F96
:103010006BEA869F612D1124669566956695F62F5D
:10302000FF5F50E0683008F05BC0862F90E0880FAB
:10303000991FEC01CC0FDD1FCC0FDD1FCC0FDD1F66
:10304000C80FD91FC40FD51FCC0FDD1FCA57DC4EC8
:103050000990D881C02DF83008F467C0DA01AA0FB2
:10306000BB1FAE57BB4E0D911C91DA01AA0FBB1FBF
:10307000A25ABB4E8D919C919801281B390BAF2F02
:10308000B0E017970E94B351600F711F811D911D11
:103090006115710521E08207910508F05CC09BEA8B
:1030A000E99F912D1124969596959695892F880FD5
:1030B000890F880F880FE81BF0E0EE0FFF1FE75A1B
:1030C000FC4EA081B1819B012C1B3D0B0E94A85698
:1030D000C80FD91FCE01DF91CF911F910F91089595
:1030E000EA01CC0FDD1FCE57DB4E0990D881C02DF1
:1030F000DA01AA0FBB1FA25ABB4E8D919C919E0173
:10310000281B390BA62FB0E017970E94B3516C0F04
:103110007D1F811D911D6115710521E082079105BB
:10312000F8F4EB01F83008F099CF8F2F90E0880F7A
:10313000991FDC01AA0FBB1FAA0FBB1FAA0FBB1F41
:10314000A80FB91FA40FB51FAA0FBB1FAA57BC4ECB
:103150006D917C91A4CF6FEF7FEF80E090E09FCFE7
:103160006FEF7FEF80E090E0EB01DCCFEF92FF921A
:103170000F931F93CF93DF9380E0E82FF0E0EE0FE3
:10318000FF1FE453FD4E118210828F5F8231A9F739
:103190001092F1121092F01280911113823009F402
:1031A0004FC0833099F1813039F0DF91CF911F9179
:1031B0000F91FF90EF9008950091CA121091CB12D9
:1031C000E0901013EE0CF12C4F2D60E08E2D1BDFE4
:1031D000EC014F2D60E080E016DF9E01281B390BCB
:1031E000EF2DF0E0EE0FFF1FE453FD4ED8010E94DB
:1031F000B35191838083F3948CE0F812E5CFDF9193
:10320000CF911F910F91FF90EF900895209110138F
:10321000A091CA12B091CB1230E00E94B3519B0131
:10322000AC01A5E5B5E10E9469569093F112809337
:10323000F012DF91CF911F910F91FF90EF900895C1
:1032400020911013A091CA12B091CB1230E00E94CD
:10325000B3519B01AC01A5E5B5E10E946956BB27BE
:1032600097FDB095AB2F9093E5128093E412909365
:10327000E7128093E6129093E9128093E8129093FC
:10328000EB128093EA129093ED128093EC129093DC
:10329000EF128093EE12DF91CF911F910F91FF906B
:1032A000EF90089520914410309145102F3F8FEFFB
:1032B000380791F0809142109091431001969093BD
:1032C0004310809342108217930730F010924310FE
:1032D0001092421081E0089580E008950F931F93AB
:1032E000CF93DF93FC018BE1DF011D928A95E9F713
:1032F00006ED14E160E070E080E89FEBC0E0D0E014
:103300001BC0BE01882777FD8095982F0E940E5321
:1033100020E030E04FE753E40E94475220E030E0E5
:1033200040E85FE30E94DC512BED3FE049E450E4CC
:103330000E9490540E94445220E030E040E85FE355
:103340000E94DC5120E030E040E05FE30E949054B6
:1033500020E03FEF4FE757E40E9490540E94E05274
:10336000F801619371938F012196C115F1E0DF0798
:1033700041F6DF91CF911F910F91089521E030E048
:1033800002C0220F331F8A95E2F7D901A095B095AC
:1033900080914B0A90914C0A8A239B2390934C0A6C
:1033A00080934B0AE0914D0AF0914E0AEA23FB23E9
:1033B000F0934E0AE0934D0A662371F0822B932B13
:1033C00090934C0A80934B0A442331F02E2B3F2BD1
:1033D00030934E0A20934D0A089524E630E040E0F1
:1033E00050E00E948D562AE030E040E050E00E941C
:1033F0008D56605D205D30E02038310588F4F9019C
:10340000EC5AF94F808180934F0A70E06038710563
:1034100070F4FB01EC5AF94F80818093500A0895B3
:103420008FEF80934F0A70E06038710590F38FEF53
:103430008093500A089590E08038910588F4FC014B
:10344000EC5AF94F808180934F0A70E06038710523
:1034500070F4FB01EC5AF94F80818093500A089573
:103460008FEF80934F0A70E06038710590F38FEF13
:103470008093500A08951F93CF93DF931FB7F8945A
:103480006DDD0E94F93D10923E1010923D10109299
:10349000261010922510CFEFDFEFD0931A10C093B3
:1034A00019101092281010922710D0931C10C0935E
:1034B0001B1010922A1010922910D0931E10C09346
:1034C0001D1010922C1010922B10D0932010C0932E
:1034D0001F1010922E1010922D10D0932210C09316
:1034E00021101092301010922F10D0932410C093FE
:1034F0002310809141108160809341100E940C1133
:10350000D0933410C09333101092361010923510AF
:10351000C0E06C2F6E5E8C2F0E94DD3FCF5FC63007
:10352000C1F7809141108E7F809341100E940C1151
:10353000809141108860809341100E940C1110927C
:103540003410109233108FEF9FEF909336108093CA
:1035500035106C2F645F8C2F0E94DD3FCF5FCC3025
:10356000C1F780914110877F809341100E940C1118
:1035700010923410109233101092361010923510B1
:103580008FEF9FEF90933E1080933D1010921A1092
:103590001092191010921C1010921B1010921E10F5
:1035A00010921D101092201010921F1010922210D5
:1035B0001092211010922410109223106C2F6A5F29
:1035C0008C2F0E94DD3FCF5FC231C1F710923E10B9
:1035D00010923D1010922610109225101092281073
:1035E0001092271010922A101092291010922C106D
:1035F00010922B1010922E1010922D10109230104D
:1036000010922F100E946C3D10924F0A1092500A97
:1036100010924C0A10924B0A10924E0A10924D0AC8
:103620001092550A5AD01FBFDF91CF911F91089574
:103630008F929F92AF92BF92CF92DF92EF92FF92C2
:103640000F93CF93DF93EC018091940F9091950F9E
:1036500084599D4081309240A0F5862E912C811492
:10366000910479F181E0881A9108A12CB12C2FEFF7
:10367000821A920AA20AB20ABA2CA92C982C88247F
:10368000C12CD12C7601CE01A0E0B0E0803E9105A6
:10369000A105B10560F4A6014C56524F9F5FAF4F94
:1036A000BF4F6627782F892F9A2F0E9400F8219606
:1036B0008FEFD81AE80AF80AC814D904EA04FB0400
:1036C00011F7DF91CF910F91FF90EF90DF90CF90A6
:1036D000BF90AF909F908F9008950F931F93CF93BB
:1036E000DF931FB7F8940CDCC091940FD091950F25
:1036F000AE0160E070E004E2069FF001079FF00D6C
:103700001124EA57FC4E80E090E021913191DA01DA
:10371000A80FB91F2D933C93029684329105A9F707
:103720006F5F7F4F4C5D5F4F6830710529F7809167
:10373000A8149091A914FE01E05EFE4F918380834E
:10374000FE01EE5DFE4F8091A6149091A714918327
:103750008083CC5DDE4FD093950FC093940F809102
:10376000AA148883E091940FF091950FCF010196F0
:103770009093950F8093940F8091AB148183E09187
:10378000940FF091950FCF0101969093950F809330
:10379000940F8091AD148183E091940FF091950F77
:1037A000CF0101969093950F8093940F8091AC1464
:1037B0008183E091940FF091950FCF010196909342
:1037C000950F8093940F8091AE148183E091940FB4
:1037D000F091950FCF0101969093950F8093940FE0
:1037E0008091AF148183E091940FF091950FCF01F8
:1037F00001969093950F8093940F8091B0148183DC
:10380000E091940FF091950F809151139091521384
:103810009093B2148093B114928381833396F09382
:10382000950FE093940F62E08CED90E001DF1FBFF5
:10383000DF91CF911F910F910895CF92DF92EF9278
:10384000FF920F931F93CF93DF9300D0CDB7DEB7D6
:1038500080910713182F110F180F1F5F8091061307
:103860008093581280913E1290913F12A091401285
:10387000B0914112892B8A2B8B2B51F460918F0DC3
:103880007091900D8091910D9091920D0E94315602
:103890000E942E5660933E1270933F128093401206
:1038A0009093411280915612181709F110935612F5
:1038B0008EE392E10E944414A0915712BB27A19578
:1038C0000CF4B095AA0FBB1F1196209146123091AF
:1038D000471240914812509149120E9473566093CA
:1038E0004A1270934B1280934C1290934D12809118
:1038F000F5129091F612A091F712B091F8128F3F45
:103900002FEF9207A207B20709F4B3C02091491321
:1039100030914A132115324008F074C04FEF5FEF29
:10392000E090C812F090C9120090121302C0F694F1
:10393000E7940A94E2F78091411390914213811524
:1039400062E0960708F4E7C09C01325080914D1365
:1039500090914E1396958795969587958115E2E0FF
:103960009E0708F489C08C0112508091141388239B
:1039700009F488C0AA27249FB12D359FC001529F0A
:10398000B00D811D9A1F349FB00D811D9A1F112407
:1039900060913F137091401380934E1290934F1299
:1039A00080915012909151126817790721F08EE39F
:1039B00092E10E946A14C801809590958E159F052A
:1039C00008F0ACC00FEF1FEF60914B1370914C13D8
:1039D00010936A120093691280916B1290916C128D
:1039E0006817790709F48CC089E592E10F900F9070
:1039F000DF91CF911F910F91FF90EF90DF90CF90CB
:103A00000C946A142091F9123091FA1240E050E0BF
:103A1000820F931FA41FB51FC0908F0DD090900DE3
:103A2000E090910DF090920DC816D906EA06FB06BB
:103A300000F1C0908F0DD090900DE090910DF0901E
:103A4000920DC81AD90AEA0AFB0AC216D306E4067E
:103A5000F50608F063CF9E2D8D2D7C2D66270E94E4
:103A6000B456F901EE0FFF1FE05EFC4F408151811B
:103A700057CF40E050E054CF00E010E080911413A5
:103A8000811178CFC901809590958E159F0508F01A
:103A900048C02FEF3FEF60913F1370914013309378
:103AA0004F1220934E12809150129091511268172C
:103AB000790741F08EE392E149835A830E946A14A8
:103AC0005A814981AA27049FB12D159FC001509F9B
:103AD000B00D811D9A1F149FB00D811D9A1F1124D6
:103AE00060914B1370914C138093691290936A12FA
:103AF00080916B1290916C126817790709F074CF5E
:103B00000F900F90DF91CF911F910F91FF90EF9049
:103B1000DF90CF90089520E030E018CF0E0D1F1DEC
:103B200053CF2E0D3F1DB7CFAF92BF92CF92DF92F2
:103B3000EF92FF920F931F93CF93DF9300D0CDB7F7
:103B4000DEB76C017B0180918513811159C0042F70
:103B5000017040FD48C0142F127041FD3CC021117E
:103B60000DC00F900F90DF91CF911F910F91FF909B
:103B7000EF90DF90CF90BF90AF900895002351F069
:103B80008091D7169091D8168C259D258C7F892BF6
:103B900009F0F1C0112329F38091D9169091DA161A
:103BA0008E259F2588279E7F892BD9F20F2D06957C
:103BB0004091AC144F70406BE0918319F0918419DF
:103BC00021E063E070E083E899E10995F092DA166C
:103BD000E092D916C6CFF092C912E092C8122A8399
:103BE0002CDE2A81BCCFD092CB12C092CA122A837B
:103BF0004983BCDA6FEF81E0C9D749812A81ABCF15
:103C000060E070E05FEFFB01EE0FFF1FE60FF71FB4
:103C1000EE0FFF1FEE0FFF1FE456F44F928599231E
:103C2000F1F0852F992787FD9095DC01AA0FBB1F26
:103C3000A80FB91FAA0FBB1FAA0FBB1FA456B44FD2
:103C400000811181228133818D919D910D90BC91D4
:103C5000A02D80179107A207B30708F4562F6F5FB6
:103C60007F4F6630710579F65F3F09F47ACF852F73
:103C7000992787FD9095FC01EE0FFF1FE80FF91FB4
:103C8000EE0FFF1FEE0FFF1FED55F44F808140FD3B
:103C900068CF41FF66CF1BEA819F112D1124169535
:103CA00016951695912F990F910F990F990F182F1F
:103CB000191BB70180E090E00E940C5320E830E02F
:103CC00040E857E30E9490546B017C01612F70E043
:103CD00080E090E00E940C5320E030E040E05FE3A1
:103CE0000E94DB519B01AC01C701B6010E94DC516F
:103CF000D62EE72EF82E092F20E030E0A9010E94F1
:103D0000405287FD55C020E030E040E451E46D2D85
:103D10007E2D8F2D902F0E941C5418162CF4D12C20
:103D2000E12C90E4F92E01E4A12EB12CAA0CBB1CCD
:103D300089E593E1A80EB91E2BEA3AEA4AEA55E46E
:103D40006D2D7E2D8F2D902F0E9490540E94E05259
:103D5000F501718360830ADA6FEF81E00F900F90B5
:103D6000DF91CF911F910F91FF90EF90DF90CF9057
:103D7000BF90AF900BC7C60190589C013595279511
:103D800035952795092F06952F7733274091AC1449
:103D90004F70406EE0918319F091841963E070E0F8
:103DA00083E899E10995D092D816C092D716F2CE41
:103DB000D12CE12CF12C00E0B7CF8091AB1487FD22
:103DC00009C06F7070E0992787FD90956817790793
:103DD00009F0089580E8289F90011124242BC9013F
:103DE000905220E041E060E070E0880F991F880F5A
:103DF000991F9ACE4F925F926F927F928F929F926D
:103E0000AF92BF92CF92DF92EF92FF920F931F93E8
:103E1000CF93DF938091A6149091A7149093010102
:103E200080930001C0900401D09005017C01EC1842
:103E3000FD08C80ED91EC0910201D091030197015F
:103E40002C1B3D0B40E050E0812C912CA12C60E814
:103E5000B62EC501B4010E94B45629013A0120933F
:103E600006013093070140930801509309018E0128
:103E70000095109598012C193D0940E050E0C501CE
:103E8000B4010E94B45649015A0120930A013093AB
:103E90000B0140930C0150930D018091DB0F909129
:103EA000DC0F08171907B8F48FEF9FE720E041E017
:103EB00060E070E0DF91CF911F910F91FF90EF9044
:103EC000DF90CF90BF90AF909F908F907F906F903A
:103ED0005F904F9029CE8C179D07C0F0AC0160E039
:103EE00070E08E159F0530F0C816D90690F080E07E
:103EF00090E0DCCFCB01BA016C1B7D0B81099109ED
:103F0000A30192010E94B9519058D0CF80E090E86F
:103F1000CDCF9A01AB012C193D0941095109C501C9
:103F2000B4010E94B95190589058C0CFCF93DF93FD
:103F3000CDB7DEB728970FB6F894DEBF0FBECDBF62
:103F400092E09D8394E09E8397E09F839CE0988716
:103F500095E0998393E09A8391E09B831C82823061
:103F6000D9F1CCF0843009F461C06CF5DB01CA01F1
:103F700081709927AA27BB2721E0822780930A1303
:103F8000427055276627772775956795579547950A
:103F900040930B1304C0882359F0813091F1289687
:103FA0000FB6F894DEBF0FBECDBFDF91CF9108955D
:103FB000440F551F661F771F809106138170842B55
:103FC00080930613ECCF853051F7FE01E40FF51F07
:103FD000818180931213E3CFDB01CA01817099279D
:103FE000AA27BB2721E0822780930C134270552714
:103FF00066277727759567955795479540931613CC
:10400000CECF809108138B7C41305105610571053D
:10401000E1F04230510561057105E9F04330510589
:1040200061057105B1F080930813B9CFFE01E40F6B
:10403000F51F85818093101328960FB6F894DEBF84
:104040000FBECDBFDF91CF91D5CE80618093081395
:10405000A6CF8460E8CF806280930813A0CF2F9210
:104060003F924F925F926F927F928F929F92AF9208
:10407000BF92CF92DF92EF92FF920F931F93CF9355
:10408000DF93CDB7DEB760970FB6F894DEBF0FBEF3
:10409000CDBF80903513909036139C868B86A09070
:1040A0002D13B0902E13BE86AD86212C312CF3C07B
:1040B00083E0EF85F88980A7CF010E94B134909109
:1040C0000B13992309F40CC183E0ED81FE8180A7D5
:1040D000CF010E94B1349091AF14992309F4FCC030
:1040E0001595812F992787FD9095019620FEFAC09E
:1040F0004FEF5FEF849F9001859F300D949F300DAF
:104100001124922F8827AC01662757FD6095762FE2
:104110008091391390913A134A015B01880E991EE0
:10412000A11CB11CD501C401B7FCF5C02091371307
:10413000309138136A017B01C20ED31EE11CF11CC1
:10414000F7FCE5C020913313309134134A015B0131
:10415000820E931EA11CB11C89829A82AB82BC8202
:10416000B7FCD0C020913113309132134A015B016A
:10417000820E931EA11CB11CB7FCC0C020912F134E
:10418000309130132A013B01420E531E611C711CF9
:1041900077FCB0C000912B1310912C13F8018A0109
:1041A0009B010E0F1F1F211D311D0F8318872987AB
:1041B0003A8737FD9AC009811A812B813C8101150C
:1041C0001105F1E02F07310524F00FEF1FEF20E07C
:1041D00030E0C982DA82EB82FC82C114D10441E072
:1041E000E406F10444F04FEF5FEF60E070E04983D4
:1041F0005A836B837C83BC01CD016115710551E04D
:104200008507910524F06FEF7FEF80E090E09FE05D
:10421000C92EE12CF12C2B853C8549815A818F8553
:1042200098890E94A6350F81188529853A85011540
:10423000110561E02607310524F00FEF1FEF20E0A4
:1042400030E0B301A2014114510481E06806710419
:1042500024F04FEF5FEF60E070E08114910491E093
:10426000A906B1042CF088248A94982CA12CB12C96
:10427000BFE0CB2EE12CF12C2D853E85B4018D8144
:104280009E810E94A635EFEF2E1A3E0AF6E02F1609
:10429000310409F444C0122D5AE2B52EB29CC0017B
:1042A000B39C900D11249C012E5B3E4E388B2F87C2
:1042B00020910C13EF85F88926A39C012A5B3F4EC1
:1042C0003E832D8390910A13F90196A390911613C2
:1042D0009111EECE81E0EDCE40E050E0BA0118CF72
:1042E00081E0F3CE41E050E005CF1F8218861986A9
:1042F0001A8661CF412C512C32014CCF812C912C4C
:1043000054013CCF19821A821B821C822BCFC12CF4
:10431000D12C760117CF80E090E0DC0107CF6096CA
:104320000FB6F894DEBF0FBECDBFDF91CF911F91C6
:104330000F91FF90EF90DF90CF90BF90AF909F9044
:104340008F907F906F905F904F903F902F90089547
:10435000CF92DF92FF920F931F93CF93DF931F9221
:10436000CDB7DEB781E00E94ED130E9464348091E6
:104370000E1381114DC00E94EC411091AD1480913B
:10438000EB0B181721F081E04ED21093EB0B10913C
:104390000F138091EA0B181731F081E044D21330EB
:1043A000A8F51093EA0B49DA5ADE0E94B618F0908D
:1043B000B0146CEBC62E62E1D62E2CE00FEF1FEF8F
:1043C00009C0F601118300832F5FF2E0CF0ED11CEC
:1043D000223191F0FF20A9F3422F60E08EE729837C
:1043E0000E940318F6019183808329812F5FF2E0F8
:1043F000CF0ED11C223171F70F90DF91CF911F9119
:104400000F91FF90DF90CF900C948A3110E0C9CFCC
:1044100061E083E593E12BD2B0CFCF93DF9320917E
:10442000AB1427FD0BC06F7070E0332727FD30956C
:104430006217730719F0DF91CF9108958091AA1444
:104440008823C9F34436B8F7C42FD0E08091A8146C
:104450009091A914C817D90771F3CE010E94DD16F7
:10446000882349F3D093A914C093A814109273130E
:1044700034D9DF91CF916CCFE82FF0E0E553F64FC0
:1044800090819170803209F456C078F0843209F43A
:104490004CC0A0F1863209F445C008F058C0909392
:1044A000041381E08093731353CF8C31C8F08C31A7
:1044B00009F444C08091E8098170909108139473C5
:1044C000892B9091E90990FD47C090E0892B90914C
:1044D000EA0990FF45C092E0892B80930813E1CF51
:1044E0008A31A8F08091E60981709091E50990FDEC
:1044F00035C090E0892B80930913D3CF8232C1F06D
:1045000018F090930013CDCF9093FE12CACF88314C
:1045100031F0893109F0089590930213C2CF90933E
:10452000FF12BFCF90930513BCCF90930113B9CF67
:1045300090930313B6CF9093FD12B3CF9091E709F8
:104540008091061390FB80F980930613AACF8732DF
:1045500011F790930E13A5CF98E0B8CF92E0CACF91
:1045600090E0BACFCF938091AA148823D1F08091A4
:10457000A8149091A9140E94DD168823C1F080919F
:10458000AA148823D9F00E94A8131092731381E013
:104590009091AA14911101C080E080937113CF9182
:1045A00008958BED90E00E94DD168111E8CF81E047
:1045B0000E9496158091AA148111E5CFC8E18C2F35
:1045C0005BDFCF5FC832D9F781E00E947840DBCF54
:1045D000CF93DF93C42FD22F8091AB1487FD0BC0F4
:1045E0006F7070E0992787FD90956817790719F02B
:1045F000DF91CF910895C11135C02091AA14D23016
:1046000008F481C02223A1F38C2F80518E3198F1C0
:104610008C2F80558E3108F04FC0EC2FF0E0EE0F5C
:10462000FF1FE958FD4E408151812D2F30E0CA0116
:1046300096958795969587958F77992782179307F3
:10464000B9F2CA0188279E7F220F331F220F331F22
:10465000822B932B9183808381E080937313DF916E
:10466000CF9176CEC13009F461C0C03409F469C07D
:104670002091AA14C7CFEC2FF0E0EE0FFF1FE950F6
:10468000FD4E808191812D2F30E0AC01452F5527C3
:1046900046954217530709F4ABCF8C7F9170322FA8
:1046A0002227330F822B932B9183808381E0809389
:1046B0007313DF91CF914CCE8C2F80538A3108F049
:1046C00097CFEC2FF0E0F0972D2F30E0DF01AC52C8
:1046D000B94F4C9187E090E0841B910902C0359559
:1046E00027958A95E2F7822FDF01A350BD4E9C915A
:1046F000291709F43EC02C93C1E0719761F1CC23D6
:1047000009F476CFA9CF622F772767FD70958D2F9B
:1047100090E06817790709F475CFD093AA140E9426
:104720006D1B20DF15DE2091AA146CCF7D2F770F33
:1047300020E042E060E080E090E0F6D92091AA1409
:1047400061CFD11104C0DF91CF910C946E3681E01E
:104750008093ED0B4DCF882371F00E940A4286E0D2
:10476000E4EEFBE0A3E5B3E101900D928A95E1F759
:10477000C6CFC0E0C2CF0E94EC41F1CF8091AE1411
:10478000813009F008956A3FB1F06C3F41F0683F15
:10479000C9F78091FB128F5F8093FB12089580917F
:1047A000EE0B823089F18091760C823059F786E7E2
:1047B0009CE00C94DA3A8091EE0B823079F1109201
:1047C000710C1092700C8FEF9FEF9093730C80938D
:1047D000720C8091760C8230E1F01092F90C1092FC
:1047E000F80C8FEF9FEF9093FB0C8093FA0C909353
:1047F000820D8093810D8FEF9FE7909343108093FC
:1048000042101092FB1208958EEE9BE00E94DA3A5D
:10481000CACF86E79CE00E94DA3ADFCF8EEE9BE0BB
:104820000E94DA3ACCCFE6EAFBE09FEFDF01129775
:104830001C921082DF0113979C93DF0114979C93C5
:10484000DF011A971D921D921D921C9213973C96A0
:104850002BE0EE3EF20751F7811101C0089580E18F
:10486000ECE8FAE0DF011D928A95E9F708951F93BD
:10487000CF93DF93182FD92FC62F8091EC0B86177B
:10488000F1F080E0D0DFC093EC0B46E050E06FEF3A
:1048900070E084EE9BE00E94CA55E12FFD2FA4EE4C
:1048A000BBE080E091919F3FB9F09D938F5F863090
:1048B000C9F71092E40BDF91CF911F91089546E064
:1048C00050E064EE7BE0812F0E94A3550097D9F65B
:1048D000DF91CF911F9108958111EBCFE4EEFBE0C2
:1048E00086E0DF011D928A95E9F7DF91CF911F9154
:1048F0000895CF93DF93FC01D62FCFB7F894218191
:1049000030E0C90101964281642F70E00E94C851D5
:10491000408150E08417950791F0A381B481A20FE4
:10492000B31FDC93818190E00196628170E00E9468
:10493000C8518183CFBF81E0DF91CF910895CFBF70
:1049400080E0DF91CF910895FC013FB7F894218179
:104950009081291728F48281820F891B3FBF089517
:10496000822F891B3FBF0895AF92BF92CF92DF92F3
:10497000EF92FF920F931F93CF93DF93082FD62EC2
:10498000C0E0D0E088E8E82E98EEC92EC00E2FE3F4
:10499000F22E1FEFEC9EF001ED9EF00D1124E2517E
:1049A000F44F8081833079F02196C230D10591F7A0
:1049B000DF91CF911F910F91FF90EF90DF90CF90FB
:1049C000BF90AF9008950C3F09F45AC00D3F09F411
:1049D0006AC00E3F09F48CC0DD2091F14091000DBA
:1049E000842F8F5F8093000D5F0161E8A60EB11CDC
:1049F000D5016C91862F90E02091FF0CDC01A20F75
:104A0000B11DA038B10584F6442309F49EC0462F99
:104A10004150242F332727FD30952E5F3F4F2E0F17
:104A20003F1FD9015E919D01752F7F73C71609F451
:104A3000BBCF57FF03C0415047FFF3CF20E88DC0E5
:104A40008091000D811177C05F0161E8A60EB11C55
:104A5000D5012C9130E02F5F3F4F2E0F3F1F40912B
:104A6000FF0C50E06EE370E0C9010E94CA558091CE
:104A7000FF0CF5019081890F80831092FF0C94CF79
:104A8000DF01AF57BF4F1C92DF01AA57BF4F1C92E7
:104A90001092FF0C319640E850E06FEF70E0CF01CC
:104AA0000E94CA5581CFDF01AA57BF4F8C9188233E
:104AB00009F47ACF81508C938091FF0C811141C011
:104AC0005F0161E8A60EB11CD5018C91882309F421
:104AD0006BCF8150D5018C939F01280F311DD901D7
:104AE00011969C91119711961C9397FF5DCFEECF75
:104AF0005F01B1E8AB0EB11CD5014C91842F90E061
:104B00002091FF0CBC01620F711D603871050CF023
:104B10004BCF9F012A573F4FD9015C915F5F5C9358
:104B20002091000D211122C0E80FF91FF1824F5F83
:104B3000F501408339CF81508093000D811134CF2E
:104B400083CF81508093FF0C2FCF9F012A573F4F77
:104B5000D9014C914F5F4C9320E0E80FF91F822F51
:104B60008C2981836F5FF50160831ECF8091FF0CDC
:104B70008F5F8093FF0C18CF211106C0472F582F4D
:104B8000692F7727CA0108950C9496142F923F92AB
:104B90004F925F926F927F928F929F92AF92BF924D
:104BA000CF92DF92EF92FF920F931F93CF93DF93F9
:104BB000CDB7DEB7A0970FB6F894DEBF0FBECDBF5E
:104BC0008C87362E882309F49BC0E0912313F09143
:104BD00024134090251350902613409117135091A1
:104BE000181380911D1390911E1320914F13309133
:104BF00050130091D90F1091DA0F20900913609192
:104C000013131093DC160093DB16F093DE16E0937B
:104C1000DD165092E0164092DF165093E216409354
:104C2000E1169093E4168093E3163093E6162093F2
:104C3000E5162092E7166093E816000F012F001F7B
:104C4000110B11951A95EE0FEF2FEE1FFF0BF1953B
:104C50005F01BA94612C712C73016201CC0CDD1CD4
:104C6000EE1CFF1CCC0CDD1CEE1CFF1CC40CD51C68
:104C7000E61CF71C73E0F694E794D794C7947A95F2
:104C8000D1F756954795569547954C01969487943C
:104C9000969487948D2D99279B878A87A52FBB276C
:104CA000BF83AE83E92DFF27F987E887D701C601C7
:104CB0009927AA27BB278B8B9C8BAD8BBE8B66233A
:104CC00009F443C0623008F430C29CE0E92EF12CB4
:104CD0008E819F81B7010E94C851AE81BF81A81B00
:104CE000B90BBF83AE83CF01B7010E94C851E81B47
:104CF000F90BF987E887188A1F861E861D862DC046
:104D00000091D90F1091DA0F8091DB169091DC168B
:104D1000E0912313F09124138017910709F4E1C166
:104D2000409025135090261340911713509118135B
:104D300080911D1390911E1320914F1330915013A9
:104D400020900913609113135CCFFA01FF27FE87AF
:104D5000ED87A4015527588B4F8750910E13598B1F
:104D60007091AF147D8F832F99279C8F8B8F3091FB
:104D7000F4123A8BE12CF12C58E15D8320E0B8016C
:104D8000882777FD8095982F69837A838B839C830E
:104D9000C501AA2797FDA095BA2F8F8B988FA98F51
:104DA000BA8FF8A2EF8E0AC02F5F4F8D58A14E5FC9
:104DB0005F4F58A34F8F263009F438C137FC02C02B
:104DC0002311F2CF8F8D98A1880F991FAF8CB8A0B7
:104DD0008A0D9B1D880F991F8457954FFC01E85E33
:104DE000FE4F3081332309F43AC1FC01E95EFE4FE6
:104DF000B080BD823D81A32EB12C48E1A41AB10838
:104E0000888499848A0C9B1C0F8D18A10A5B1F4E05
:104E1000F801EA57FD4FC080D180EE24D7FCE09422
:104E2000FE2C69817A818B819C81C60ED71EE81E7B
:104E3000F91E8E819F818A0D9B1D97FD27C1422FF0
:104E40006D852E8F0E940318C80ED91EE11CF11C1F
:104E50002E8DF7FC29C1C114D10471E0E706F104DD
:104E60002CF0CC24CA94DC2CE12CF12CF801EE5669
:104E7000FD4F40805180662457FC6094762C8981D8
:104E80009A81AB81BC81480E591E6A1E7B1E4F89D8
:104E9000588D698D7A8D440E551E661E771E422FE1
:104EA0004A5FC40197FCFDC06F852E8F0E940318D6
:104EB000480E591E611C711C2E8D77FCEEC04114EA
:104EC000510451E0650671042CF044244A94542C9A
:104ED000612C712C8A859B85222051F061E0261679
:104EE00009F4F2C08A859B858A0D9B1D97FDF6C04B
:104EF000422F445F6B892E8F0E940318F801E256FF
:104F0000FD4F80809180AA2497FCA094BA2C880E33
:104F1000991EA11CB11C2E8DB7FCBBC0811491043D
:104F200081E0A806B1042CF088248A94982CA12C46
:104F3000B12C3989311104C05D8D552309F451C05C
:104F4000822F8595992787FD9095019620FF9BC01C
:104F50006FEF7FEF869FA001879F500D969F500DAA
:104F600011246B8D7C8D469FC001479F900D569FED
:104F7000900D1124AA2797FDA095BA2FC80ED91E0F
:104F8000EA1EFB1EF7FC9CC0C114D10471E0E706C9
:104F9000F1042CF0CC24CA94DC2CE12CF12C480E2A
:104FA000591E6A1E7B1E77FC87C041145104E1E044
:104FB0006E0671042CF044244A94542C612C712CFC
:104FC000880E991EAA1EBB1EB7FC72C081149104E4
:104FD000F1E0AF06B1042CF088248A94982CA12C1F
:104FE000B12CAA88F801AA2009F43EC0EE5AFD4F60
:104FF000D182C082F801E25AFD4F51824082F8010D
:10500000E659FD4F918280822110CECEF801EA5BF5
:10501000FD4F91828082C8CE6091E7162612B7C0FC
:10502000609113137091E8166713EBCDA0960FB63D
:10503000F894DEBF0FBECDBFDF91CF911F910F91CE
:10504000FF90EF90DF90CF90BF90AF909F908F90A8
:105050007F906F905F904F903F902F9008953C8588
:105060003F3F09F0A1CEC6CEE25DFD4FD182C082A6
:10507000F801E65CFD4F51824082F801EA5BFD4F8A
:105080009182808291CE61E070E064CF80E090E018
:10509000D6CE812C912C540141CF412C512C320180
:1050A0000ECF80E090E000CFC12CD12C7601D3CE82
:1050B000812C912C54018ACF412C512C320175CF77
:1050C000C12CD12C760160CFB7FC34C0B594A79425
:1050D0008A859B858A0D9B1D97FF0ACF80E090E013
:1050E00007CF8091DD169091DE16409025135090E9
:1050F0002613E817F90709F017CE8091DF16909173
:10510000E016409117135091181348165906B1F044
:1051100080911D1390911E1320914F1330915013C5
:1051200020900913609113136CCD188A1F861E8678
:105130001D8613CE7FEFA71AB70AC8CF8091E1165C
:105140009091E2164817590719F780911D13909115
:105150001E132091E3163091E4168217930749F04D
:1051600020914F1330915013209009136091131325
:1051700048CD20914F13309150136091E5167091F6
:10518000E616209009132617370709F445CF6091DA
:10519000131337CDCF92DF92EF92FF92CF9390917E
:1051A000FF1220910213992309F492C040911B131E
:1051B00050911C1360E070E0222309F485C0C09078
:1051C0002113D0902213E12CF12C8823A1F09923F4
:1051D00081F08091081385FD0CC08091541290914C
:1051E0005512AA2797FDA095BA2F480F591F6A1F7D
:1051F0007B1F211172C0CFB7F8944115510521E0F2
:105200006207710524F04FEF5FEF60E070E0DB01B3
:10521000CA0177FD77C00E94940E46EC41BB469AC6
:1052200031E035B921E428B950EF5BB992EA9EB973
:1052300087E881BB00C000C041BB469A35B928B998
:1052400060E76BB99EB981BB00C000C041BB469A04
:1052500035B928B95BB99EB981BBD701C601C11464
:10526000D10421E0E206F10424F08FEF9FEFA0E0EB
:10527000B0E0B7FD43C00E94940E46EC41BB469A95
:1052800031E035B927E428B950EF5BB992EA9EB90D
:1052900087E881BB00C000C041BB469A35B928B938
:1052A00060E76BB99EB981BB00C000C041BB469AA4
:1052B00035B928B95BB99EB981BBCFBFCF91FF90FB
:1052C000EF90DF90CF900895C12CD12C76017DCF47
:1052D0004FEF5FEF60E070E06FCF8091081384FDC7
:1052E0008ACF8091541290915512AA2797FDA095CC
:1052F000BA2FC80ED91EEA1EFB1E7DCF80E090E0BB
:10530000DC01B9CF80E090E0DC0185CF86EC81BB89
:10531000469A15B896E898B993E09BB91EB897E8F5
:1053200091BBEFE9FFE03197F1F700C0000081BBCE
:10533000469A15B823E828B923E12BB922E02EB903
:1053400091BBFAE0FA95F1F700C081BB469A20EED6
:1053500027B997E09AB92DB915B820E828B99BB9B3
:105360001EB897E491BB92E09A95F1F700C096B110
:1053700099B19CB181BB479A87EE87B987EF8AB90B
:1053800082EE8DB9EAE0EA95F1F700C008951F9327
:10539000CF93DF93D82FD86F86958695869528E092
:1053A00030E001C0220F8A95EAF7C22FC095CD23C5
:1053B0001FB7F894CB010E94940EE6ECE1BB469A2D
:1053C0003D2F330F367031649D2F96959270906A01
:1053D00071E075B938B9A0EFABB99EB967E861BBA8
:1053E00085E08A95F1F70000E1BB469AFC2FFF0F9C
:1053F0004C2F46955C2F551F5527551F8F2F8670B4
:10540000582B5064C0718F2F880F80728C2BF07CCA
:105410008F2B4270406A75B958B98BB94EB961BBD0
:105420008AE08A95F1F700C0E1BB469A75B938B9B0
:10543000ABB99EB961BB8AE08A95F1F700C01FBF86
:10544000DF91CF911F9108952F923F924F925F92DB
:105450006F927F929F92AF92BF92CF92DF92EF9224
:10546000FF920F931F93CF93DF93CDB7DEB7CD5548
:10547000D1090FB6F894DEBF0FBECDBF882309F463
:1054800008C3512C352C330C330C330CE6EC4E2E68
:10549000CC24C394D12CCC0EDD1E9E01255F3F4F42
:1054A00069963FAF2EAF69974FB7F89441BA469AC5
:1054B000952D990F292F26702064892F880F8072CF
:1054C000907C892B952D9695927031E035B928B94D
:1054D0008BB99EB987E881BB5DE05A95F1F7000072
:1054E00041BA469A80EE87B997E09AB98DB935B935
:1054F00080E488B91BB88EB987E481BB62E06A9505
:10550000F1F700C026B199B18CB141BA479A622E29
:10551000669473E06722A0E82A9F90011124622A12
:10552000292F2071622A292F269526952870622A14
:1055300096959076692A90E0880F991F8470992734
:10554000682A87EE87B987EF8AB982EE8DB94FBF97
:10555000732C912C66E0262E7FE7A72EB12C09C074
:105560008250808366949394739488E0981609F42B
:10557000D0C0072D10E0F801E553F64F8081982F39
:105580009E7F71F7962D91708170981759F3892F2E
:105590008A608083BFE3B71508F473C0E92EFF2447
:1055A000E7FCF094872D6E969FAF6E970E943C2289
:1055B0006E969FAD6E97E114F10409F4C9C0872D72
:1055C0008051823008F4F4C1FAE07F1609F4DFC19B
:1055D0003BE08091870D731609F411C2882309F40A
:1055E000B7C05DE07512F6C061E09091860D911133
:1055F00060E00E941E3991E0EF2809F4B8C0809164
:10560000DA0980FF14C1A9E0A71508F076C1B2E15C
:105610007B1609F404C6ECE07E1609F458C1FDE0DF
:105620007F1609F416C290917113953009F419C1CF
:10563000992309F431C279E0771508F498C09230C3
:1056400009F47FC308F4DDC2953008F090C0809162
:105650007213B72DAAE08A9FB00D11248B2FB0933F
:105660007213943009F452C5992787FD90950E94D2
:10567000DD1681112DC4EFEFE09372130E94B22268
:1056800076C0492F552747FD509580918013811191
:1056900071C08091811381116DC0452B51F08091B3
:1056A000EE0B813009F4CFC28091760C813009F481
:1056B000BFC24091870D4111EBC0172D1852809148
:1056C000EE0B833009F457C18091760C833009F4D6
:1056D00052C18091FC1221E040E050E8692F810F17
:1056E0006E969FAF6E970E94B6368091FC12810F26
:1056F0006E969FAD6E979111BAC140E4682F80916C
:10570000AC140E948E1266949394739488E098125D
:1057100030CF5394380E9FE0951508F0C5CEC35A8C
:10572000DF4F0FB6F894DEBF0FBECDBFDF91CF9134
:105730001F910F91FF90EF90DF90CF90BF90AF90AF
:105740009F907F906F905F904F903F902F90089523
:1057500067E2761609F454C0E114F104F1F53FE074
:10576000731609F447C090E0EF2809F048CF0E9473
:10577000A821F8CE452B09F4F5CEEEEEF6E0D601E1
:105780008AE001900D928A95E1F76996AEADBFADC2
:105790006997E22D1D92EA95E9F7872D8855809348
:1057A000FC128093FE0C8093840D4AE050E0BE0111
:1057B000665F7F4F992787FD90950E943A56C601F4
:1057C0000E94821380918013882309F4CBCE10921B
:1057D0008113C8CE27E27216B1F07EE0771681F110
:1057E0005FE07512C0CF80918113882309F4B3C0A4
:1057F00010928113909380138FEF80938313B3CF14
:10580000E114F104D1F00E940A42E4EEFBE0A3E5CA
:10581000B3E1822D01900D928A95E1F78091AA144F
:105820008111A1CF8BED90E00E94CF439CCFB2E1DC
:105830007B12F1CE0E943B1A9ACF0E94EC41E5CF39
:105840008091AA14882309F4EECE809171138823E5
:1058500009F412C11092711390917113953009F0EF
:10586000E7CE8091EE0B833029F08091760C833067
:1058700009F07DCF32E0371508F479CFF801E05E0A
:10588000F84F80818F3F09F472CF61E06DD86FCF00
:10589000272D20549111BEC08091860D882309F4D4
:1058A0008FC1413009F420C3E1E0FDE080E090E0E9
:1058B00005C001968038910509F454CE4191241316
:1058C000F8CFFC01EF5FF24F206820834BCE809130
:1058D000AA14811106C08BED90E00E94CF43809105
:1058E000AA1491E0811190E09093AA140E946D1B7C
:1058F0000E94B2220E94A8213ACF109282131092E5
:10590000811382E2EEEFF6E0DE01D39601900D9274
:105910008A95E1F780918313871509F418C2709274
:10592000831384E0781609F49DC3871508F072C1CB
:10593000E8E07E1609F4EAC1E71508F4BAC2F5E01A
:105940007F1609F474C326E0721211CF84E199E046
:105950000E9482130CCF80918213882309F490C097
:105960001092821381E080938113909380138FEFC4
:1059700080938313F8CE692F812F6E969FAF6E9719
:105980000E94B424C7D46E969FAD6E97A2CE81E0DC
:105990002091870D213009F449C16091860D6E96E2
:1059A0009FAF6E970E941E396E969FAD6E97D4CEB4
:1059B00081E0E1E17E1280E028E8829FF00111247D
:1059C000E251F44F2081213081F008F4EDC0223003
:1059D00009F45DC1233009F0FBCD21E04091AA1408
:1059E000442309F463C12093711362E06E969FAF64
:1059F0006E970E9458426E969FAD6E97E5CD8230AD
:105A000009F42DC108F4C4C0833009F434C18111F4
:105A1000AACEA2CEA1E0BDE0FD0105C03DE0E13887
:105A2000F30709F4FCC181918F3FC1F3413009F4C0
:105A300030C180E090E005C001968038910509F4FE
:105A400091CD4D914F3FC1F7FC01EF5FF24F2083A5
:105A500089CD9111E8CD80917113823009F465C12F
:105A6000843009F462C182E08093711380CE60E0DB
:105A700070E80E94751276CD81E080937113D3CDCA
:105A80008FE380938213909380138FEF809383131F
:105A90006ACEA8E05A2EF6CC60917F1359E05715D4
:105AA00008F465CE272D671509F404C1462F552744
:105AB00047FD5095872D992787FD90950A964817A1
:105AC000590709F44DC270927F138FEF9FEFDC01ED
:105AD00080937B1390937C13A0937D13B0937E13DC
:105AE000822F992787FD90958C01000F111F080FB9
:105AF000191F000F111F000F111F005E1A4F0E9487
:105B0000A813D80112966D917C911397C6010E943B
:105B1000DC55F60101900020E9F73197CF018C198F
:105B20009D092DE330E240E0208331834283F80178
:105B30002081213009F48EC108F031C1E2E0F0E0AB
:105B4000EC0FFD1FE80FF91F1082D8011196EC91A0
:105B5000EE0FFF0BE95EFC4E8081918190937A13EA
:105B600080937913A0E0B0E080937513909376133F
:105B7000A0937713B0937813C6010E94821380918B
:105B8000AA148111F4CD8BED90E00E94CF43EFCDAC
:105B90006091860D83E06E969FAF6E970E941E39CE
:105BA0006E969FAD6E97D8CD20917113223009F477
:105BB0006BC220918013222309F417CF61E016CF26
:105BC000413009F45CC1E1E0FDE080E090E004C018
:105BD00001968038910541F041912413F9CFFC01E1
:105BE000EF5FF24F5FEF5083E1E0FDE081918F3F87
:105BF00009F0B8CC7DE0E138F707C1F70E9402391F
:105C0000B1CC913009F0B3CD7092721383E08093E0
:105C10007113ADCD91E0791609F45BC0791608F0E7
:105C20003CC181E699E00E948213A1CD80E0B5CE0F
:105C300062E06E969FAF6E970E9458426BD36E964D
:105C40009FAD6E9736CD62E080E06E969FAF6E9707
:105C50000E9458425FD36E969FAD6E9725CD60919E
:105C6000860D80E06E969FAF6E970E941E396E96ED
:105C70009FAD6E9771CD6091860D82E06E969FAF5D
:105C80006E970E941E396E969FAD6E9765CD60E04F
:105C9000ADCE822F90E0FC01EF5FF24F2083F50143
:105CA000E81BF90BEF5FF24F20835CCC20E02093E0
:105CB00071139BCE265F20937F138FEF9FEFDC0144
:105CC00080937B1390937C13A0937D13B0937E13EA
:105CD00007CF8091AB14F60162E08602E00DF11D62
:105CE000112464A975A9C6010E94DC55D6010D9046
:105CF0000020E9F71197E6EDF8E0822D01900D9272
:105D00008A95E1F7C6010E94821331CD8091AE14CD
:105D1000813009F4F6C1823009F47AC2811127CDAD
:105D200080E399E00E94821322CD81E09091AA1431
:105D3000911101C080E0809371132FEF20937213B3
:105D400016CD7092721384E08093711310CDE4E04D
:105D50007E1609F450C2E71508F4D7C0F1E07F16AB
:105D600009F42AC27F1608F4BFC122E0721609F4B2
:105D700033C233E07312D3CD8091DB0F9091DC0FEF
:105D80009093A7148093A6140E946D1B0E94FA1E84
:105D900085EB98E00E94821370928313E8CC223046
:105DA00009F0EACE8AE1EDEFF2E1A9EEB6E1019069
:105DB0000D928A95E1F76D961CAE1DAE1EAE1FAE1C
:105DC0006D976A96FFAC6A976D964CAD5DAD6EAD02
:105DD0007FAD6D97F80181810E94961F4AE150E0E6
:105DE0006DEF72E189EE96E10E94A355009709F4E8
:105DF0009EC16D966CAD7DAD8EAD9FAD6D976F5FA5
:105E00007F4F8F4F9F4F6D966CAF7DAF8EAF9FAF23
:105E10006D97643071058105910599F6ADCE80913D
:105E2000AE14EFEFFFEFF093820DE093810D81113F
:105E3000FDCD8091EE0B823009F4F8CD8091760C87
:105E4000823009F4F3CD8FEF9FE790934310809356
:105E50004210ECCDE181FF27E7FDF095E350FD4EC8
:105E6000E081F0E03296EE0FFF1FE00FF11F60813E
:105E7000718102968C0D9D1D0E94DC557DCE822F76
:105E800090E0FC01EF5FF24F6FEF6083F501E81BDC
:105E9000F90BEF5FF24F6083A7CEA2E07A1609F408
:105EA000A9C0B3E07B1263CC82EE98E00E9482131B
:105EB0005ECC39E0731609F465C052E1751257CC17
:105EC00081E0909185139111DDC0809385134FCCB3
:105ED00080917213992787FD90959093A9148093D0
:105EE000A8140E946D1BC7CB822F90E0FC01EF5FCE
:105EF000F24F208120682083F501E81BF90BEF5F4A
:105F0000F24F8081806880832DCB56E0751609F4AE
:105F10001BC1751608F4D5C068E0761609F43BC1BC
:105F200079E07712FCCC81E09091AF14911101C01F
:105F300080E09091B014911170C190E0890F90E0D1
:105F40000196AC01417055274093AF148370992797
:105F500086958093B0140E946D1B0E94A821DFCC0F
:105F6000262F2A5020937F138FEF9FEFDC01809321
:105F70007B1390937C13A0937D13B0937E136213D5
:105F8000AFCDF5CB88E0EDE4F9E0D60101900D92BC
:105F90008A95E1F78091AF14811183C08FE696E670
:105FA000A6E6B0E088879987AA87BB87D6010D90BF
:105FB0000020E9F7CD0101978C199D09D601A80FA2
:105FC000B91F2CE0E5E5F9E001900D922A95E1F783
:105FD0002091B014F601E80FF91F222309F49EC0A6
:105FE0008FE69EE6A0E083879487A587C6010E947E
:105FF0008213BDCB8091AC14F60172E08702E00DF4
:10600000F11D112464A975A9C6010E94DC55D601B1
:106010000D900020E9F71197ECEDF8E0822D01904A
:106020000D928A95E1F7C6010E948213A0CB2091C0
:1060300084138091AD1490E0022E02C0959587954F
:106040000A94E2F780FD34C088E0ECE0F9E0D60184
:1060500001900D928A95E1F72F5C2B83C6010E9477
:10606000821385CB86E593E6ADE2B0E089839A831F
:10607000AB83BC83809184138F5C8B83C6010E94A9
:10608000821375CB80E021CF63E06E969FAF6E9751
:106090000E94584285E0809371136E969FAD6E9773
:1060A00093CA8FE69EE6A0E088879987AA877ECF6D
:1060B00087E0E5E0F9E0D60101900D928A95E1F7DD
:1060C000CBCF81E090E00090841302C0880F991F2D
:1060D0000A94E2F79091AD1498279093AD140E9422
:1060E0006D1B0E94A8211BCC81E00E94961581E0C7
:1060F0008093731381E799E00E9482130E94A82184
:106100004BCE89E399E00E94821331CB992787FD1A
:1061100090950E94CF4380917213A6CA8FE696E6AF
:10612000A6E6B0E083879487A587B6875FCFF8019E
:106130002F2D32E02302E00DF11D112464817581C1
:10614000C6010E94D15518CD67961FAE1EAE679747
:1061500000E010E005C00F5F1F4F0436110591F0FD
:10616000C8010E94DD168823B1F3BE016B5A7F4F30
:10617000C8010E94A41667968EAD9FAD67970E94D6
:106180008041E9CF87EC98E00E9482130E94B222FE
:106190000E94A82101CE8091AE14992787FD909589
:1061A000019663E070E00E94C8518093AE140E9493
:1061B0006D1B0E94A821B3CB8091AB14992787FD5A
:1061C0009095029661E170E00E94C85181508093E1
:1061D000AB140E946D1BA3CB8091AC14992787FD53
:1061E000909501968F70907897FD27C08093AC149E
:1061F0000E946D1B94CB80918413992787FD909505
:10620000019666E070E00E94C8518093841387CBAA
:1062100083E499E00E948213AACA92E08FCE109282
:1062200082131092811382E2EEEFF6E0DE01D39644
:1062300001900D928A95E1F772CB0197806F9F6F65
:106240000196D4CF0F931F93CF93DF938091DB0FF1
:106250009091DC0FE0910001F0910101A091040107
:10626000B091050160910201709103019B0120959D
:1062700030952817390740F42FEF3FE7C901DF9128
:10628000CF911F910F9108958617970748F18C01C0
:1062900020E030E0EF01CA1BDB0B8C179D07C0F438
:1062A000A9019801261B370B41095109609106018C
:1062B0007091070180910801909109010E94B951E4
:1062C0009C013058C901DF91CF911F910F91089522
:1062D000EA0FFB1FE817F90758F020E030E0CECFB7
:1062E00020E030E8C901DF91CF911F910F9108950F
:1062F000A90198012E1B3F0B4109510960910A0128
:1063000070910B0180910C0190910D010E94B95187
:106310009058D6CFCF92DF92EF92FF921F93CF93F8
:10632000DF931F92CDB7DEB78091EE0B833009F477
:1063300096C08091760C833009F493C080917113DC
:10634000882309F4D0C0813009F4FEC08091721313
:1063500087FDF5C060E2805D0E941B1A40E06091FD
:10636000AA1484E00E94BE1980917113811164C047
:1063700061E08091AA14882309F45EC040E086E0C1
:106380000E94BE198091EE0B41E0823009F4A7C053
:1063900061E0811101C060E080E00E94BE1980913F
:1063A000760C41E0823009F498C061E0811101C0AF
:1063B00060E081E00E94BE1961E08091870D81302C
:1063C00009F060E040E082E00E94BE198091870DF4
:1063D00041E0823009F040E061E0823008F460E0A2
:1063E00083E00E94BE1960918513462F88E00E94C9
:1063F000BE19409181138091801361E0811103C027
:10640000411101C060E087E00E94BE198091870DB4
:10641000811114C08091EE0B833081F08091760C55
:10642000833061F08091711361E0823019F0843023
:1064300009F060E0462F08C060E0A0CF8091860D93
:106440008823F1F161E040E085E00F90DF91CF918A
:106450001F91FF90EF90DF90CF900C94BE19809128
:10646000760C21E030E0833011F020E030E048E8A5
:10647000429FC001439F900D11248251944FFC0113
:10648000EA57FF4F1081FC01EF57FF4F20818091A9
:10649000FF0C90E0820F911D41E0803891050CF4D3
:1064A00040E0612F70E080E090E049830E94ED19A8
:1064B00049811436B0F4642F89E00E94BE194ECF92
:1064C0008091EE0B61E0833009F4BDCF8091760CB2
:1064D000833009F4B8CF60E0B6CF40E066CF40E04B
:1064E00057CF61E0E9CF40E060E089E00E94BE194B
:1064F0008091751390917613A0917713B0917813D2
:10650000B7FD1DC0109174131031F1F12091791372
:1065100030917A1340E050E0A4E6B0E00E94695662
:106520006C01FF24D7FCF094EF2C812F0E949D1763
:10653000811116C0C701B6010E94ED190FCF60E2AC
:1065400080E20E941B1A0ACF6091A8147091A914CE
:1065500080E090E00E94ED1940E060917313ACCFB1
:1065600082E3C81AD108D7FC19C0EE24D7FCE09406
:10657000FE2C60917A136095661F6627661F40E0C7
:1065800089E00E94BE19D6CF5DDE9C01442737FD0D
:106590004095542F30584F4F5F4FBECFD194C19488
:1065A000D108E3CFFC0126893789468D578DAA276C
:1065B000429FB12D539FC001349FB00D811D9A1F82
:1065C000529FB00D811D9A1F112480A391A3409565
:1065D0005095AA27429FB12D539FC001349FB00D03
:1065E000811D9A1F529FB00D811D9A1F112482A3F5
:1065F00093A340855185628573854083518362836F
:1066000073830895FF920F931F93CF93DF93EC0151
:10661000F62E1C821D821E821F820E891F896CA18C
:106620007DA1CB01A0E0B0E077276627980140E08C
:1066300050E00E94B4563F8F2E8FF11019C084E0B5
:1066400089A719A218A2B801C9010E9485149BA3A9
:106650008AA388899989AA89BB8988839983AA830F
:10666000BB83FFA2DF91CF911F910F91FF900895FF
:1066700081E089A7CE0196DFFFA2DF91CF911F9124
:106680000F91FF900895CF93DF93EC011C821D8240
:106690001E821F82188219821A821B8289A58F5F2F
:1066A00089A7833061F1853021F1823019F0DF91C3
:1066B000CF9108956E897F897DA36CA38C899D8974
:1066C0000E94851499A388A36E897F898C899D89EE
:1066D000809590950E9485149BA38AA34C855D8527
:1066E0006E857F85488359836A837B83DF91CF9151
:1066F000089519A61DA21CA2DF91CF91089519A299
:1067000018A28E899F899BA38AA3DF91CF910895B8
:10671000CF92DF92EF92FF92CF93DF93EC01CC8088
:10672000DD80EE80FF808F2D9927AA27BB27892B3C
:106730008A2B8B2B09F042C089A5823009F433C023
:1067400070F5813009F444C040E050E02AA13BA13B
:10675000AA27429FB12D539FC001349FB00D811DC8
:106760009A1F529FB00D811D9A1F112428A139A193
:10677000820F931F9DA38CA3488159816A817B81DD
:106780004C0D5D1D6E1D7F1D4C835D836E837F836D
:10679000DF91CF91FF90EF90DF90CF9008958330FD
:1067A000A1F0843089F68EA1811122C0BB27AF2DC4
:1067B0009E2D8D2DAC0140955095C8CFCE0163DF45
:1067C000CC80DD80EE80FF80B7CF4C895D89BECF65
:1067D0008EA1811105C077276F2D5E2D4D2DB6CF6F
:1067E00040E253E0C701B6010E949614AC01AECF5F
:1067F00040E251E0C701B6010E949614DBCFCF936F
:10680000DF93E4EAFBE0A6EABBE080E090E05AE236
:106810006FEF11C0589F9001599F300D1124E9016D
:10682000CE5BDE4E49A5411127C001963C961C96D1
:1068300086309105F1F02081222361F3589FE00119
:10684000599FD00D1124CE5BDE4E29A52111EDCF2D
:1068500010821C92EF0121976883EF0122976883D1
:1068600020812223B9F201963C961C968630910530
:1068700011F7DF91CF9108951FA21DA21CA21C82C7
:106880001D821E821F821F8E1E8E19A619A218A29B
:106890001BA21AA2188219821A821B82E901CA5B02
:1068A000DF4E1FA21DA21CA21C821D821E821F82FF
:1068B0001F8E1E8E19A619A218A21BA21AA2188238
:1068C00019821A821B82B1CF809141108E7F9091E4
:1068D000FD1291118160809341100E940C118091F2
:1068E0004110877F9091001391118860809341102F
:1068F0000E940C11809141108D7F9091FE12911198
:106900008260809341100E940C11809141108F7E13
:106910009091011391118061809341100E940C119C
:10692000809141108B7F909103139111846080932B
:1069300041100E940C11809141108F7D90910413A1
:1069400091118062809341100E940C11809141103E
:106950008F7B9091051391118064809341100C946A
:106960000C11CF93DF93EC01898D90E09927FC0106
:10697000E45BFE4F3491FC01E45BFD4F2491FC018C
:10698000E45BFC4F849190E0A0E0B0E0DC0199274B
:106990008827922B28A5832B022E04C0B695A79595
:1069A000979587950A94D2F7880F991FAA1FBB1F46
:1069B000880F991FAA1FBB1F880F991FAA1FBB1FF3
:1069C000880F991FAA1FBB1F88879987AA87BB8733
:1069D0004B8D50E05527FA01E45BFE4F8491FA019C
:1069E000E45BFD4F9491FA01E45BFC4F449150E06D
:1069F00060E070E0BA0155274427592B482B022E3E
:106A000004C076956795579547950A94D2F7440F39
:106A1000551F661F771F440F551F661F771F440FB2
:106A2000551F661F771F440F551F661F771F4C8722
:106A30005D876E877F874D8D50E05527FA01E45BB7
:106A4000FE4F8491FA01E45BFD4F9491FA01E45BFF
:106A5000FC4F449150E060E070E0BA0155274427B4
:106A6000592B482B04C076956795579547952A95DD
:106A7000D2F7440F551F661F771F440F551F661F1F
:106A8000771F440F551F661F771F440F551F661F42
:106A9000771F488B598B6A8B7B8B89A58230A9F134
:106AA00070F4813009F44EC019A218A21BA21AA2D8
:106AB000188219821A821B82DF91CF910895833048
:106AC000B9F0843089F719A218A26E897F898E8D5A
:106AD0009F8D0E9485149BA38AA388899989AA897E
:106AE000BB8988839983AA83BB83DF91CF91089563
:106AF00019A218A28E899F899BA38AA31882198242
:106B00001A821B82DF91CF9108956E897F898C89CB
:106B10009D890E94851499A388A36E897F898C8999
:106B20009D89809590950E9485149BA38AA38C854E
:106B30009D85AE85BF8588839983AA83BB83DF91BA
:106B4000CF910895CE01DF91CF912CCDCF92EF92CE
:106B5000FF920F931F93FC01AC2DA078C0FE08C0DC
:106B6000808D918D8617970719F0718F608FA1E046
:106B7000C1FE08C0828D938D8417950719F0538F3D
:106B8000428FA1E0C2FE08C08489958982179307CD
:106B900019F0358B248BA1E0C3FE08C0848D958D40
:106BA0008017910719F0158F048FA1E0C4FE0EC065
:106BB000868997898E159F0549F0F78AE68ACF0165
:106BC0001F910F91FF90EF90CF90CBCEA111F7CFF7
:106BD0001F910F91FF90EF90CF900895AF92BF92C9
:106BE000CF92EF92FF920F931F93CF93DF93F62EE6
:106BF000142F590180E00E94ED13612F81E00E9463
:106C0000C625002309F45BC08091870D811157C010
:106C1000FF2009F44AC02091471330914813A50181
:106C2000AA27429FB12D539F7001349FB00DE11CE4
:106C3000FA1E529FB00DE11CFA1E112420953095CA
:106C4000E20EF31E5AE21502E001112420E1C22EE9
:106C500000E010E020E030E040E050E060E070E074
:106C6000CE018A5B9F4E72DF20914513309146130F
:106C7000A501AA27429FB12D539F7001349FB00DEB
:106C8000E11CFA1E529FB00DE11CFA1E1124209542
:106C90003095E20EF31E20E030E040E050E060E08E
:106CA00070E0CE018E5B9E4E51DFDF91CF911F9140
:106CB0000F91FF90EF90CF90BF90AF9008954AE270
:106CC0001402E00111246F2DCE018A5B9F4E9ADCE5
:106CD0006F2DCE018E5B9E4E95DC9ACFAF92BF9208
:106CE000CF92DF92EF92FF920F93CF93DF931092A8
:106CF000ED0B33E2A32E37E0B32E45EAE42E4BE052
:106D0000F42E56EAC52E5BE0D52EE5014C2F4A192C
:106D100089919091EB0B892341F0F70180818823C1
:106D200021F0F60180818823A1F0FCE0EF0EF11C38
:106D30008CE0C80ED11CE7E0C932DE0739F7DF91DD
:106D4000CF910F91FF90EF90DF90CF90BF90AF90D9
:106D50000895F701359720813181F701329700E0DE
:106D600060E080813BDFF7011082DFCF2F923F92FE
:106D70004F925F926F927F928F929F92AF92BF924B
:106D8000CF92DF92EF92FF920F931F93CF93DF93F7
:106D9000CDB7DEB72C970FB6F894DEBF0FBECDBFD0
:106DA000782E642E552E298386958695869590E0BB
:106DB000E72DE770F0E0ED5DF84F2081FC01E4572E
:106DC000F54F662309F4C6C08081822B8083E72DAE
:106DD000F0E0EE0FFF1FE456F54F40835183412C46
:106DE000C0908F0DD090900DE090910DF090920D8D
:106DF0008091EC0B882309F409C16091EA0B6623AA
:106E000059F1272D30E080E090E02817390701F193
:106E1000E82FE695E695E695F0E0E457F54F4081DA
:106E20004423B1F0FC01E770FF27ED5DF84F50817E
:106E3000542371F0821793071CF4613009F471C078
:106E4000281739071CF4623009F46BC044244394BA
:106E5000019680389105C9F640E084EEA82E8BE0BB
:106E6000B82E11E0872C912CD5018D915D018F3FBB
:106E700009F457C0242E332427FC30949101220FAB
:106E8000331F220D331D220F331F220F331F2457B0
:106E9000354FF901E85EFE4F1083F901E75EFE4FC2
:106EA0001083F901E65EFE4F1083F901EC5EFE4FA0
:106EB00060825182F901EA5EFE4F7082F401E80FB0
:106EC000F11DCF01F901E95EFE4F8083F901E05F1A
:106ED000FE4FC082D182E282F382F901E55EFE4F6D
:106EE00029812083042D262D352D61E077DE209128
:106EF000EB0B04C0242E332427FC3094C1010196EF
:106F000066E070E00E94C851482FFC01ED5DF84F2B
:106F10008081822379F35AEEA5165BE0B50609F06D
:106F2000A3CF2C960FB6F894DEBF0FBECDBFDF9176
:106F3000CF911F910F91FF90EF90DF90CF90BF9076
:106F4000AF909F908F907F906F905F904F903F9009
:106F50002F90089520958081282320830091EA0BAB
:106F600080E090E06FE770E0023009F44BC09C01D4
:106F7000122FE22FE695E695E695F0E0E457F54FFF
:106F80004081442321F1F901E770FF27ED5DF84FBF
:106F900050815423E1F0E4EAFBE04081442339F0DE
:106FA000DF0112974C9150E04217530781F03C9655
:106FB000ABE0EC3EFA0789F7F901EE0FFF1FE4564C
:106FC000F54F60805180712E4424439409CF01967F
:106FD0008038910549F676EAE72E7BE0F72E10E03F
:106FE000F70132978081882331F0F701349780814F
:106FF000871509F4A5C01F5FFCE0EF0EF11C1630E9
:1070000079F78FCF9B01281B390BB2CF2091EB0B67
:1070100003E217E04CE95BE05B834A8394EA292EA4
:107020009BE0392EF8014FEF88248A94982C540164
:10703000302F1DC06D917D918D919C916C157D05BA
:107040008E059F0538F4C1010197DC018C917816FB
:1070500009F4D6C06A817B81645F7F4F7B836A833A
:107060007CE0270E311C87E0E932F807C1F05E2F83
:10707000531B8191822371F3D1018C91AA81BB8131
:107080008111D8CF6D917D918D919C916815790575
:107090008A059B05F8F64B015C01452FDBCF842F59
:1070A0004F3F09F0DACE62EA262E6BE0362EE3E29D
:1070B000F7E088248A94982C54019E2F931B4191C9
:1070C000422301F1D1015C91A52FA695A695A69525
:1070D000B0E0A457B54F4C91411121C0A1014650D9
:1070E0005109DA014D915D916D917C914A835B83E9
:1070F0006C837D83481559056A057B0518F44A01A0
:107100005B01892FBCE02B0E311C47E0E932F4070C
:10711000A1F68F3F39F187FD04CF482F9ECE5770DF
:10712000A52FB0E0AD5DB84F5C915423B9F2BCE03F
:107130002B0E311C47E0E932F40709F0BECFE9CF4E
:10714000F70110828091ED0B811155CF319710829C
:10715000F701339700E0262D352D412F60E0808127
:107160003DDD49CF5091EA0B5A87E3EAFBE07B868D
:1071700088248A94982C54018E829F82A886B9868E
:1071800025C01F0147E0241A3108D1018D909D9040
:10719000AD90BC908A829B82AC82BD824E815F8121
:1071A0006885798584169506A606B70648F48A810F
:1071B0009B81AC81BD818E839F83A887B9878C8595
:1071C0003C9697E00932190709F4A5CF902E931A3F
:1071D0009C86D8019D918D01922391F3BA85B1309F
:1071E00051F078F2B23061F790816B85961740F7D5
:1071F0008C859B87E5CF90815B855917C8F3E0CFDD
:10720000452F2BCECF938091830D8F3FA9F0C82FB0
:10721000CF778091850D8C0F20E040E050E060E05A
:10722000885EA4DD6091850D6C0F685E40E0809102
:10723000AC14CF910C948E12CF9108959F92AF927F
:10724000BF92CF92DF92EF92FF920F931F93CF9353
:10725000DF93182F962E8091870D811709F443C074
:10726000D1DF8FEF9FEF9093820D8093810D8FEF91
:107270008093830D40E850E06FEF70E081E09DE087
:107280000E94CA5533E2A32E37E0B32E45EAE42E1E
:107290004BE0F42E57EAC52E5BE0D52EE5014C2FCE
:1072A0004A1989919091EB0B892341F0D7018C9178
:1072B000882321F0F601808181115BC0BCE0EB0ED8
:1072C000F11CECE0CE0ED11CF7E0C932DF0739F734
:1072D00080E1ECE8FAE0DF011D928A95E9F710926F
:1072E000ED0B111116C0911004C08091860D811113
:1072F00029C01093870D9092860DDF91CF911F9139
:107300000F91FF90EF90DF90CF90BF90AF909F9044
:1073100008952091AE148FEF9FEF9093820D80938C
:10732000810D2111E0CF8091EE0B8230E1F280914E
:10733000760C8230C1F28FEF9FE7909343108093D9
:107340004210D1CFA1E0BDE0FD019FEF05C0319615
:107350008DE0E138F80749F0808187FFF8CF90830E
:10736000F6CFEDE0A138BE0799F08D918F3FC9F3BC
:10737000C0CF379720813181F601349700E060E07B
:1073800080812CDCD7011C92F6013197108296CFB8
:1073900039DFAFCF0F93CF934FB7F89436EC31BBB3
:1073A000469A80EE87B997E09AB98DB981E085B9A0
:1073B00080E488B91BB880E28EB987E481BB52E0D3
:1073C0005A95F1F700C026B199B18CB131BB479AFB
:1073D000C22FC695C37050E8259F90011124C22B7F
:1073E000292F2071C22B292F269526952870C22B74
:1073F00096959076C92B90E0880F991F84709927F5
:10740000C82B87EE87B987EF8AB982EE8DB94FBF57
:1074100080910E13882381F080917F18C5FF2FC0C3
:107420008C2785FD0EC08091AE148230C1F0C093D0
:107430007F18CF910F91089580917F188C2785FF39
:10744000F2CF8091870D882339F161E0C5FD60E0BE
:10745000F5DE0E948A318091AE14823041F7C0FF80
:10746000E6CF80917F1880FDE2CF8091FB128E5F86
:107470008093FB12C0937F18CF910F91089585FFE1
:10748000CFCFC8D786E0E4EEFBE0A3E5B3E10190FF
:107490000D928A95E1F7C7CFC5FF11C01FDC00E050
:1074A0004091AC144F70406BE0918319F0918419B6
:1074B00020E463E070E083E899E10995B4CF81E0CE
:1074C0008093ED0B0FE7ECCFCF938091870D88234E
:1074D00099F0E1E0FDE004C08DE0E138F80761F0EB
:1074E00081918F3FC9F38EDE8091870D8230E1F06C
:1074F000833019F1813009F1CF91089561507109FC
:107500008109910960687F6F8F6F9F6F6F5F7F4FF9
:107510008F4F9F4FFB017093820D6093810DEF5F42
:10752000F24F80818F3F21F50E942E566F7777278B
:107530008827907897FFEECFE1CF2091810D309191
:10754000820D07C09C01FC01EF5FF24F40814F3F6D
:1075500059F4C90101968F77907897FFF3CF01977F
:1075600080689F6F0196EECF8093810D9093820D7E
:10757000C081CF778091840D885E20E040E050E8A4
:1075800061E08C0FF3DB8091840D885E60E070E831
:107590008C0F0E947512E091810DF091820DEF5FCA
:1075A000F24F80818093830D8091840D8093850DAF
:1075B000CF910895BF92CF92DF92EF92FF920F93F7
:1075C0001F93CF93DF938C017C0181E8E80EF11CBF
:1075D000F70180818823B9F1E801CC57DF4F88811A
:1075E000998197FD30C0F801E80FF91F818168018A
:1075F000F7E8CF0ED11C22C078E1B72EB80EF60105
:107600008081B80E20E040E050E060E08B2DAEDBE2
:1076100040E06B2D8091AC140E948E12888199817C
:107620000196F701608170E00E94C85199838883B8
:10763000F801E80FF91F818187FF05C08F73982F2C
:107640009E539230C8F6DF91CF911F910F91FF901A
:10765000EF90DF90CF90BF9008958F929F92AF925E
:10766000BF92CF92DF92EF92FF920F931F93CF932F
:10767000DF931F92CDB7DEB700E010E0F8E8BF2E31
:10768000B09E4001B19E900C11248EEE9BE0880EBE
:10769000991ED4018C91823099F00F5F1F4F0230F8
:1076A000110571F70F90DF91CF911F910F91FF900E
:1076B000EF90DF90CF90BF90AF909F908F90089504
:1076C0006401B1E8CB0ED11CF6018081882329F337
:1076D0007401F2E8EF0EF11CD701ED91FC91E80D79
:1076E000F91D41814E33B1F0C401498363DF498103
:1076F000842F8E53823070F0F401EC57FF4FD70186
:107700002D913C91318320838091FE0CF401E95747
:10771000FF4F80834F73842F8E53823088F0E8E1CF
:10772000AE2EA40E8091FE0CA80E20E040E050E8A2
:1077300061E08A2D1BDB60E070E88A2D0E947512E3
:10774000F701808191810196D6016C9170E00E94D1
:10775000C85191838083F401E80FF91F418147FDEF
:10776000D9CF9BCF842F2091AB1427FD09C06F7018
:1077700070E0332727FD30956217730709F00895ED
:1077800020E040E050E060E0F1CA842FE091AB14CB
:10779000E7FD09C06F7070E0FF27E7FDF0956E17F9
:1077A0007F0709F00895422F50E0542F4427550FCA
:1077B00041505E4F61E0211101C060E020E0D6CA77
:1077C0006F928F929F92AF92BF92CF92DF92EF9281
:1077D000FF920F931F93CF93DF93E091A319F09142
:1077E000A419309719F083E899E109958BE69AE19D
:1077F0000E94A424082F10E00115110509F478C097
:10780000C0E0D0E090916B1A20916D1AEE24E394C1
:10781000F12CE3E09E2EF4E08F2EA2E0AA2EBB24F2
:10782000B394892F622F90E070E00E94C851E091DC
:107830006E1AF0916F1AE80FF91FF081F83F08F007
:1078400065C0F7FF71C08091A819843031F0F093C2
:10785000A519F092AA19E092A9198F2F807F803B79
:1078600079F198F4803961F1803A51F1803841F131
:10787000F03F09F4B1C0F73F09F4C3C01092A81952
:107880001092AA191092A9191DC0803D09F4A1C037
:1078900008F49CC0803EA1F0803F51F7EF2FE15FDC
:1078A000EF3030F7AE2FB0E0A15BB84F8C91813054
:1078B00009F49BC0E8F2823009F48BC08330F1F602
:1078C0009092A8193FB7F89490916B1A892F90E085
:1078D000019620916D1A622F70E00E94C851982F76
:1078E00080936B1A3FBF2196C017D10708F499CF38
:1078F000DF91CF911F910F91FF90EF90DF90CF908C
:10790000BF90AF909F908F906F900895D090A819DE
:10791000B092A81920E040E06F2F81E090E00E9433
:10792000A112D092A819CECF6090A819662051F26A
:107930004091A9195091AA199A01ABEABAEA0E949A
:10794000A8566C01D694C794C601880F991F8C0D58
:107950009D1D6A01C81AD90AD601AD57B64E929636
:10796000FC93CA0101969093AA198093A91921E06A
:10797000C216D104B9F022E0C216D10409F0A2CF98
:107980002091A7194091A6196091A5190E94A112F2
:107990008091A819843009F495CFF092AA19E09249
:1079A000A91990CF22E062128DCF20E04091A61954
:1079B0006091A5190E94A1128091A819843009F440
:1079C00081CFD092AA19C092A9197CCF803C09F02E
:1079D0004FCFA092A81976CF8092A819F093A5193D
:1079E000F092AA19E092A9196DCF8093A81920E00E
:1079F00040E06F2F81E090E00E94A1121092A81940
:107A000061CF4091A9195091AA199A01ABEABAEA3B
:107A10000E94A856969587959C01220F331F280F28
:107A2000391FDA01A21BB30BAD57B64E9296FC93E9
:107A3000CA0101969093AA198093A9192091A719B8
:107A40004091A6196091A5190E94A1121092A8193F
:107A500039CFCF93C82F6C2F88E89DE00E947924FE
:107A600081110FC088E89DE00E94A424882399F327
:107A70000E9453126C2F88E89DE00E94792488238D
:107A800089F3CF910895EF92FF920F93CF93DF93F5
:107A90001F92CDB7DEB77B016115710539F40F90E8
:107AA000DF91CF910F91FF90EF900895842F29835C
:107AB000D0DF298182E0E816F10488F3822FC9DF44
:107AC000E2E0EE16F10459F3802F0F90DF91CF9191
:107AD0000F91FF90EF90BDCF6F927F929F92AF92E8
:107AE000BF92CF92DF92EF92FF920F931F93CF93AB
:107AF000DF931F92CDB7DEB711E0612E10E1712E3A
:107B000060E008E010E086ECC82EDD24D39490EF0E
:107B1000B92E27E8E22EF301819191913F01B8EF50
:107B2000FB2EF62A262F269526952695A80102C01B
:107B3000440F551F2A95E2F7942E90949F20AFB6DC
:107B4000F89469830E94940EC1BA469A3F2D330F70
:107B5000367031649F2D96959270906AD5B838B979
:107B6000BBB89EB9E1BA55E05A95F1F70000C1BA29
:107B7000469A792D770F492D4695592D551F552732
:107B8000551F872F8670582B5064292D2071872F01
:107B9000880F8072822B707C872B4270406AD5B828
:107BA00058B98BB94EB9E1BA8AE08A95F1F700C0AD
:107BB000C1BA469AD5B838B9BBB89EB9E1BAEAE0BD
:107BC000EA95F1F700C0AFBE69816F5F603209F0DE
:107BD000A2CF0F90DF91CF911F910F91FF90EF9067
:107BE000DF90CF90BF90AF909F907F906F900C945C
:107BF0000C11CF93DF9310924F0A1092500A1092FB
:107C00004C0A10924B0A10924E0A10924D0A109292
:107C1000550A40E061E088E00E94BE1910923810D9
:107C20001092371059DF2FEF82E597E02150804006
:107C30009040E1F700C00000C1E4D0E188818E7F70
:107C400088830E940C1188818D7F88830E940C118B
:107C50008881877F88830E940C1188818F7E88832A
:107C60000E940C1188818F7D88830E940C1188816D
:107C70008F7B88830E940C1188818B7F88830E9470
:107C80000C1110923E1010923D1010923A1010926A
:107C900039101092401010923F1010923210109232
:107CA000311010923C1010923B1060E383E00E9470
:107CB000321160E783E00E94321162EB83E0DF91D2
:107CC000CF910C9432116091930D663090F06C302E
:107CD00040F06B5D86E60E941B1A81E00E94FF0F58
:107CE000FBCE655D82E60E941B1A81E00E94FF0FB9
:107CF000F3CE6F5C81E60E941B1A81E00E94FF0FA9
:107D0000EBCECF92DF92EF92FF92CF93DF93D82FFB
:107D1000C9E1D9DFC150E9F710928118109280189B
:107D20006AE081E10E9478110E945C11C12CD12C83
:107D3000760134C060E082E00E94781161E088E062
:107D40000E94781180E00E94A81160E181E00E9409
:107D5000781181E00E94A81160E080E10E94781112
:107D600080E00E94FF1160E180E00E94781160E0F5
:107D700080E10E94781181E00E94FF116AE080E0BA
:107D80000E947811D1500E945C11C80ED91EE11CCE
:107D9000F11C99DF80918218853058F4D111CACF37
:107DA000B601C701DF91CF91FF90EF90DF90CF90A8
:107DB0000895CC24CA94DC2C7601F2CF2F923F9206
:107DC0004F925F926F927F928F929F92AF92BF92EB
:107DD000CF92DF92EF92FF920F931F93CF93DF9397
:107DE000CDB7DEB72D970FB6F894DEBF0FBECDBF6F
:107DF000682E6C83542E1092821870E080E090E020
:107E00000E940C539B01AC0160E070E080E090E4C4
:107E10000E94F35424EA30ED42E851E40E94905469
:107E20009B01AC0160E074E284EF99E40E94475248
:107E30001B01482E9983862D90E09F838E832C8191
:107E4000235081E090E0022E01C0880F0A94EAF7E7
:107E50008D837EE0772E00E010E8EE24EA94FE2C7D
:107E6000AE81BF81AA0FBB1FAF5FBF4EBB83AA838A
:107E7000E22FFF27E1950CF4F0954F01AA2497FC1F
:107E8000A094BA2CFD86EC860AC0EC85FD85E00F37
:107E9000F11FFD87EC87169507957A9431F1462DF1
:107EA00060E0852D0E9403182C853D85821793077D
:107EB00008F44EC06FEF7FEF8FE79FE7262F372F35
:107EC000482F592FF980622D732D842D9F2D0E94EC
:107ED000405287FDDACF2C853D85201B310B3D8735
:107EE0002C87169507957A94D1F6EC84FD848C81C5
:107EF00090E0880F991FFC01EE0FFF1FEE0FFF1F90
:107F0000EE0FFF1FE80FF91F8E819F81E80FF91F09
:107F1000EE0FFF1FEA57FC4EF182E08280E02D96C3
:107F20000FB6F894DEBF0FBECDBFDF91CF911F918A
:107F30000F91FF90EF90DF90CF90BF90AF909F9008
:107F40008F907F906F905F904F903F902F9008950B
:107F5000AA81BB812D933C938D81D3DE6B017C0183
:107F60006F3FBFEF7B078B079B0729F1C501B4016A
:107F70000E940E539B01AC0160E070E080E090E451
:107F80000E94F354562F472F382F292FC701B601CF
:107F90002B873A87498758870E940C535885498513
:107FA0003A85F32E2B85E22F252F342F4F2D5E2F70
:107FB0000E94905483CF8FEFB2CF0F931F93CF9334
:107FC000DF93182F8093930DC62FD0E02296DE0109
:107FD000AA0FBB1FA350B04F2FEF3FEF2D933C9341
:107FE0008C3008F062C003E04CE0602F812FE6DEA9
:107FF000811103C00F5F0730B9F7E12FF0E0DF0117
:10800000AA0FBB1FAE50BC4E4D915C91CA01880FA8
:10801000991FDF01AA0FBB1FAA5EBB4E2D913C9199
:10802000821B930BDF01AA0FBB1FA253BC4E8D9383
:108030009C939C01220F331F241B350BDF01AA0FD9
:10804000BB1FA655BC4E2D933C93220F331FDF015F
:10805000AA0FBB1FAA57BC4E281B390B2D933C936C
:10806000AF01440F551F4E575B4ECF01880F991F2C
:10807000825A9B4EDC018D919C91880F991FEE0FC7
:10808000FF1FE65CFB4E20813181821B930BFA01BE
:1080900091838083CC0FDD1FC350D04F198218828B
:1080A000DF91CF911F910F9117CD04E044E2602F33
:1080B000812F84DE811103C00F5F0830B9F7E12FF3
:1080C000F0E0EE0FFF1FEA5EFB4E43E0DF01949706
:1080D00020813181220F331F84A195A1281B390BE8
:1080E00011963C932E934150FD014F3F79F7D2CF2B
:1080F0003F924F925F926F927F928F929F92AF9238
:10810000BF92CF92DF92EF92FF920F931F93CF9384
:10811000DF93CDB7DEB768970FB6F894DEBF0FBE1A
:10812000CDBF082F30907413C090970FD090980F48
:10813000E090990FF0909A0F80910E0190910F01AD
:1081400020911201309113014090100150901101C3
:108150005201A094B094AC01421B530B5E834D833B
:10816000A20160E070E04F83588769877A87409169
:1081700014015091150160911601709117014B8700
:108180005C876D877E874901880E991EB40180E067
:1081900090E06F87788B898B9A8B809118019091F2
:1081A0001901A0911A01B0911B018B8B9C8BAD8B97
:1081B000BE8B9091731310E0632C772467FC70944E
:1081C000C982DA82EB82FC8275011EC0F301EE0FD8
:1081D000FF1FE554F04FC080D1800E949D17882377
:1081E00039F0EC14FD0408F051C0CC24CA94DC2C06
:1081F000EF89F88DEE0FFF1FE95EFC4ED182C08241
:1082000091E01F5F1E3119F1A12EB12CB88EAF8AFB
:10821000F501EF5CF84F80818F3F99F3011131C078
:108220008315A1F2E82FFF27E7FDF09549815A81D8
:108230006B817C81082E04C076956795579547958C
:108240000A94D2F740FDC3CF1F5F1E31E9F6909329
:10825000731368960FB6F894DEBF0FBECDBFDF91E3
:10826000CF911F910F91FF90EF90DF90CF90BF9033
:10827000AF909F908F907F906F905F904F903F90C6
:108280000895E82FFF27E7FDF095A1CFC414D5048A
:10829000D0F0C601A0E0B0E0AD80BE80CA14DB041F
:1082A000A8F49C01AD01AF80B884C984DA842A198E
:1082B0003B094C095D096B857C858D859E850E94F7
:1082C000B9516C0195CFC12CD12C92CF8C149D0447
:1082D00020F0C12C90E8D92E8BCF9C01AD01AF844A
:1082E000B888C988DA882A193B094C095D096B8965
:1082F0007C898D899E890E94B95190586C0178CFF4
:10830000BF92CF92DF92EF92FF920F931F93CF9382
:10831000DF938C01BFB6F8940150110915950795AC
:10832000159507950F5F1F4F80EF93DB80E091DB82
:1083300081E68FDB86E18DDB81E08BDB1016110699
:108340008CF5C0E0D0E0FE01EE0FFF1FEE0FFF1F27
:10835000E751F94EC080E180D280F3808C2D8F7779
:1083600078DB8E2D8F7775DB8D2D8F7772DB8F2DE0
:108370008F776FDB9D2D9295969594703E2D32955B
:10838000369536953270932B2F2D22952870922B8F
:108390008C2D881F8827881F892B5BDB2196C017AF
:1083A000D1078CF287EF55DBBFBEDF91CF911F91D4
:1083B0000F91FF90EF90DF90CF90BF9008958823AA
:1083C00049F088E89DE00E94A424811101C008952D
:1083D0000C945312F5D9F5CFCF93DF9300D000D092
:1083E00000D0CDB7DEB786E0EBE2F7E0DE01119614
:1083F00001900D928A95E1F760E0CE0101960E940E
:10840000372426960FB6F894DEBF0FBECDBFDF919E
:10841000CF910895CF93DF9300D000D000D0CDB797
:10842000DEB746E050E06FEF70E0CE0101960E94AB
:10843000CA5540E080E090E00AC02981321B3083B9
:108440004F5F46303CF501968038910519F1382F81
:10845000E82FE695E695E695F0E0E457F54F2081A4
:10846000222389F3FC01E770FF27ED5DF84F50816F
:10847000522349F3E1E0F0E0EC0FFD1FE40FF11DA2
:1084800047FDFA9580834111D8CF41E001968038AD
:108490009105E9F661E0CE0101960E943724269607
:1084A0000FB6F894DEBF0FBECDBFDF91CF91089518
:1084B0006F927F928F929F92AF92BF92CF92DF92F4
:1084C000EF92FF920F931F93CF93DF931F92CDB73D
:1084D000DEB7C62EE82EFF24E7FCF094282F38E8FC
:1084E0002303800111240251144FD8018C91681785
:1084F000E9F09091EE0BDD24D394923029F0909125
:10850000760C923009F0D12C882301F1833009F4E4
:1085100009C1823009F43BC1B2E0CB1609F455C061
:10852000E3E0CE1609F4E4C0D801CC920F90DF91BD
:10853000CF911F910F91FF90EF90DF90CF90BF9060
:10854000AF909F908F907F906F9008955801BFEFEC
:10855000AB1ABB0A9FB6F89461E0C70188539F4FDE
:108560000E941516882309F404C13801E1E86E0E53
:10857000711CE091940FF091950F8191F093950FFC
:10858000E093940FD5018D935D01A615B705A9F76A
:108590009FBEF3011082D801AA57BF4F1C9280E002
:1085A00006C08F5FF3018083803809F4B5CFF801EE
:1085B000E80FF11D918197FD03C02C912F5F2C9343
:1085C0009F3F79F7B2E0CB12ABCFC090AE1488E8F2
:1085D0008E9DF0018F9DF00D1124E251F44F8081AA
:1085E000823009F4D8C028E82E9DC0012F9D900D3F
:1085F00011248251944FFC01EE57FF4F11821082DB
:10860000FC01EC57FF4F2FEF3FEF31832083CC204D
:1086100009F473C082E0F801808380914410909146
:108620004510DD2009F482CF8F3FBFEF9B0709F48F
:108630007DCF969587952091421030914310281751
:10864000390708F073CF3801E1E86E0E711CD301D1
:108650008C91882309F46ACF7801B2E8EB0EF11C03
:10866000D701ED91FC91E00FF11F21812E33B9F07C
:10867000C80129830E94DA3A2981822F8E538230E1
:1086800070F0F801EC57FF4FD7018D919C919183C9
:1086900080838091FE0CF801E957FF4F80832F7390
:1086A000822F8E53823090F088E1D82ED20E8091A6
:1086B000FE0CD80E20E040E050E861E08D2D0E94D5
:1086C000B63660E070E88D2D0E947512F70180814A
:1086D00091810196D3016C9170E00E94C851918301
:1086E0008083F801E80FF91F218127FDD8CF1ECF25
:1086F0001092FF0CD801CC9219CF8091EE0B8230F2
:1087000009F488CF8091760C823009F483CF809170
:10871000870D81117FCF8FEF9FE790934310809358
:10872000421078CF4801FFEF8F1A9F0ABFB6F89426
:108730000E948017E091940FF091950FC8018F5718
:108740009F4FD4012D914D012083E091940FF09122
:10875000950F3196F093950FE093940FA817B907F2
:1087600081F761E0C70188539F4F0E94181BBFBE6D
:10877000D3CE9FBE40E850E06FEF70E0C5010E948D
:10878000CA5531E8632E712C600E711E02CFC801EC
:108790000E94DA3AC1CEC8010E94DA3A24CFEF92A1
:1087A000FF921F93CF93DF9300D0CDB7DEB71FB7F3
:1087B000F89489839A830E948017E091940FF09136
:1087C000950F40E09A818981A42FB0E0AA0FBB1FCA
:1087D000A95EBC4E2D913C91219331934F5F49315D
:1087E00099F7E093940FF093950F2091161320932F
:1087F0000D1320E0A22FB0E0A350BD4E3C9130837A
:10880000E091940FF091950F3196F093950FE093CE
:10881000940F2F5F273171F7A42FB0E0AA0FBB1F71
:10882000A95EBC4E2D913C91219331934F5F4E3107
:1088300099F7E093940FF093950F209114132083F0
:10884000E091940FF091950F9F012F5F3F4F309370
:10885000950F2093940F209115132183E090940F8E
:10886000F090950F2FEFE21AF20AF092950FE09236
:10887000940FE3E5F3E12191D7012C93E090940F5D
:10888000F090950FBFEFEB1AFB0AF092950FE09274
:10889000940F23E1E935F20771F7209151133091DC
:1088A00052133093B2142093B114B701E9E5F3E108
:1088B00041915191DB014D935D93BD01B3E1E137EE
:1088C000FB07B1F7D7015896B093950FA093940F7B
:1088D00061E00E94181B1FBF0F900F90DF91CF9196
:1088E0001F91FF90EF9008952F923F924F925F92C9
:1088F0006F927F928F929F92AF92BF92CF92DF92B0
:10890000EF92FF920F931F93CF93DF93CDB7DEB714
:10891000CD59D1090FB6F894DEBF0FBECDBF803F51
:1089200051F1873FA9F020918D0D30918E0D2639A0
:10893000F1E03F070CF047C0A9014F5F5F4FF9011D
:10894000E751F94E808350938E0D40938D0D21C0D9
:108950008091E916813009F4B2C0811139C080914B
:10896000EA16813609F4B3C310928E0D10928D0D64
:108970000E94A8210EC010928E0D10928D0D86E9D6
:1089800091E0E9EEF6E1DF019C011D9221503040BB
:10899000E1F7C356DF4F0FB6F894DEBF0FBECDBF71
:1089A000DF91CF911F910F91FF90EF90DF90CF90CB
:1089B000BF90AF909F908F907F906F905F904F90FF
:1089C0003F902F90089541E050E020E030E0B7CF95
:1089D0008E3751F68091EB16883031F68091EC1687
:1089E000813011F680918D0D90918E0D86399140D8
:1089F00009F0BACF00E017E179E5E72E73E1F72E31
:108A0000D12C19C02BEA3AEA4AEA55E4692D7A2DAD
:108A10008B2D9C2D0E9490540E94E052D7016D93A3
:108A20007C930D5F1F4FD394B2E0EB0EF11CE0E896
:108A3000DE1609F499CFF8013197C080D8017C90F7
:108A4000F80132976081BBE0BD1558F370E080E01B
:108A500090E00E940C534B015C01672D70E0E0E850
:108A6000CE9E600D711D112480E090E00E940C5399
:108A700020E030E048EC5BE30E9490549B01AC01A5
:108A8000C501B4010E94DC51962EA72EB82EC92E26
:108A900020E030E0A9010E94405287FD15C320E08C
:108AA00030E040E451E4692D7A2D8B2D9C2D0E94FD
:108AB0001C5418160CF0A6CF6FEF7FEFAFCF80914C
:108AC000EA16823009F050CF80918D0D90918E0D75
:108AD000839709F049CF8091EB16843608F044CF94
:108AE000EDEEF6E1DE01AB58BF4F8D01208160E174
:108AF000269F90011124BF0161507109DB019C91F7
:108B00009F70922BD8019D938D013296B7E1ED3085
:108B1000FB0761F7EB96EFADEB972E2F229526958D
:108B200026952370EC967FADEC97972F9F70990F49
:108B3000990F922B392F330F330F20E06901C09426
:108B4000D094EA966FADEA97962E9694990C990C6C
:108B5000E996BFADE9979B2F969596959695BB2480
:108B6000B394B622B294BB0CA0EEBA22B92ABB0CC5
:108B7000BB0C661F6627661F9E2F9F73990FF92EE9
:108B8000F62AE12CE0E8FE1AE6966FADE697962FFE
:108B9000990FC456DF4F9883CC59D040CE57DF4F42
:108BA0002880C258D040922D9E7FC356DF4F9883B5
:108BB000CD59D04072957F70ED969FADED9717E03F
:108BC000A12EA922A29400EFA022A72AE92FE695C0
:108BD000E695E695EE967FADEE97972F917092957C
:108BE000990F907E9E2B990F990FE72FEE0FEE0FA6
:108BF0001E2F187700E01058F72FF295F695F770B2
:108C0000EF967FADEF97E72FE170EE0FEE0FEE0FCF
:108C1000EF2BF0E0E25AF84FA081CA56DF4FA8834D
:108C2000C659D040872E8694829440EF8422F72F35
:108C3000F295F695F770C158DF4F7881CF57D04045
:108C4000E72FE170EE0FEE0FEE0FEF2BF0E0E25AA0
:108C5000F84FA081C956DF4FA883C759D040E72FEE
:108C6000E695EF70F0E0E25AF84FA081C856DF4F6A
:108C7000A883C859D040729576957770C058DF4F59
:108C8000A881C058D040EA2FE170EE0FEE0FEE0F32
:108C9000E72BF0E0E25AF84F7081C756DF4F788338
:108CA000C959D0407A2E7694729450EF75227A2F5B
:108CB000729576957770CF57DF4FA881C158D04015
:108CC000EA2FE170EE0FEE0FEE0FE72BF0E0E25A25
:108CD000F84F7081C656DF4F7883CA59D040EA2FCB
:108CE000E695EF70F0E0E25AF84F7081C556DF4F1D
:108CF0007883CB59D040661F6627661FE796EFAD95
:108D0000E797FE2FF770FF0FF62B7F2F770F770F68
:108D1000770F60E02B01F0E85F1A7E2F771F77272F
:108D2000771FE8966FADE897FFE36F2E6622660C1B
:108D3000672A660C3E2E36947CE337226295669550
:108D400066956370B770BB0FBB0FB62BE0E1BE9F9B
:108D5000B0011124C957DF4F79836883C758D040C9
:108D6000A295A695A770E22DE170EE0FEE0FEE0F23
:108D7000EA2B60E070E029F07E2F770F770F60E03C
:108D80007054CC57DF4FF881C458D0404F2F4170FA
:108D9000C757DF4F4883C958D040F1FB552750F9DA
:108DA000C657DF4F5883CA58D040CD57DF4FE881B0
:108DB000C358D0404E2F4170C557DF4F4883CB5822
:108DC000D040F3FB552750F9C457DF4F5883CC5898
:108DD000D040F4FB442740F9C357DF4F4883CD58B8
:108DE000D040E1FB552750F9C257DF4F5883CE588A
:108DF000D040F2FB442740F9C157DF4F4883CF589A
:108E0000D040F5FB552750F9C057DF4F5883C05964
:108E1000D040F6FBFF27F0F9CF56DF4FF883C1595A
:108E2000D040E4FB442740F9CE56DF4F4883C25977
:108E3000D040E6FB442740F950E0440F551FE7FBC4
:108E4000552750F9550F550F542BE5FB442740F992
:108E5000542BE3FB442740F9CD56DF4F4883C359D9
:108E6000D040E2FF03C242E0242ECC57DF4F4881BE
:108E7000C458D04047FB442740F9CC56DF4F4883C5
:108E8000C459D0404FB7CB56DF4F4883C559D04067
:108E9000F89444E7EDEFF2E1DE01119601900D92B6
:108EA0004A95E1F7C757DF4F4881C958D0404093F2
:108EB000FD12C657DF4F4881CA58D0404093FE127A
:108EC000C557DF4F4881CB58D0404093FF12C4575D
:108ED000DF4F4881CC58D04040930013C357DF4F39
:108EE0004881CD58D04040930113C257DF4F48818D
:108EF000CE58D04040930213C157DF4F4881CF581E
:108F0000D04040930313C057DF4F4881C059D04031
:108F100040930413CF56DF4F4881C159D04040934E
:108F20000513CE56DF4F4881C259D04040930613F7
:108F30001092071350930813CD56DF4F5881C35931
:108F4000D040250E2092091310920A1341E040935D
:108F50000B1310920C13CC56DF4F5881C459D040DC
:108F600050930E1310920F1353E05093101340932D
:108F7000111352E05093121340931313409316139E
:108F80001092171390921813D0921A13C0921913BB
:108F900010921B13C456DF4F4881CC59D0404093E8
:108FA0001C1310921D13B0921E13309320132093A4
:108FB0001F1310922113C356DF4F5881CD59D04053
:108FC00050932213F0922413E0922313109225134E
:108FD000A0922613109227139093281310932A130C
:108FE0000093291310922B13CA56DF4F9881C6594C
:108FF000D04090932C1310922D1380922E13109228
:109000002F13C956DF4F2881C759D0402093301302
:1090100010923113C856DF4F3881C859D040309371
:10902000321310923313C756DF4F4881C959D040CD
:1090300040933413109235137092361310923713F5
:10904000C656DF4F5881CA59D040509338131092FA
:109050003913C556DF4F9881CB59D04090933A13BE
:1090600050923C1340923B1310923D1360923E137A
:1090700010923F1330924013C957DF4F2881398136
:10908000C758D04030934213209341137093441338
:109090006093431310924613109245131092481395
:1090A0001092471390E07BDB84E7FE013196ADEF31
:1090B000B2E101900D928A95E1F7CB56DF4F3881EE
:1090C000C559D0403FBF50CC60E070E0A7CC809144
:1090D000EB16863109F048CC8091EC168130E1F036
:1090E000823009F041CC8091ED16CB57DF4F1982C9
:1090F0001882C558D040843608F036CCBE016B5774
:109100007F4F90E00E94A416CB57DF4F8881998152
:10911000C558D040F5D828CC80918D0D90918E0DFA
:10912000049765E070E00E94C851C957DF4F79830A
:109130006883C758D04077FD9BC0ADEE8A2EA6E16C
:109140009A2EBEEEAB2EB6E1BB2E1FEEC12E16E15F
:10915000D12E00EFE02E06E1F02E1B01220C331C75
:10916000220C331C260E371E49E0240E311C04E06D
:1091700010E094E0492E512CF9EE6F2EF6E17F2E8F
:10918000600E711E44E050E0B301C2018751994E58
:109190000E94B955D30114962C91B0E82B9FC001C1
:1091A0001124F4019081982B9083922F92709295C4
:1091B000990F990F907CD5018C91982B9C93922FAD
:1091C00094709295990F907EF6018081982B9083F0
:1091D000822F88708295807FD7019C91892B8C93F8
:1091E000B4E04B0E511C0B5F1F4FE4E08E0E911C40
:1091F000F4E0AF0EB11C24E0C20ED11C34E0E30E4B
:10920000F11C0215130509F0B7CFC957DF4F2881AC
:109210003981C758D0402E5F3F4F220F331F220F96
:10922000331FE090ED16FFB6F894E4E9FDE040E06E
:1092300052E0DF01BA011D9261507040E1F78901EF
:10924000055011092EEE36E1A801B901CF010E94A7
:10925000B0550C56124F1093950F0093940F61E088
:109260008E2D90E00E94181BFFBE7ECB212CFDCDE1
:1092700024E030E0D6CFEF92FF920F93CF93DF93AD
:109280001F92CDB7DEB77B0160918D0D70918E0D71
:109290006115710529F0E61AF70A81E0E81AF1086C
:1092A000E114F10439F40F90DF91CF910F91FF9009
:1092B000EF900895842F298317DB2981E2E0EE16D1
:1092C000F10488F3822F10DBF2E0EF16F10459F37A
:1092D000802F0F90DF91CF910F91FF90EF9004CBF3
:1092E0001F920F920FB60F9211240F900FBE0F9086
:1092F0001F9018951F920F920FB60F9211240F9086
:109300000FBE0F901F9018951F920F920FB60F92DD
:1093100011240BB60F922F933F934F935F936F934C
:109320007F938F939F93AF93BF93CF93DF93EF93ED
:10933000FF9334997CC0CFB7F89456EC51BB469A52
:1093400070EE77B967E06AB97DB915B8D0E8D8B9D9
:109350006BB91EB8B7E4B1BB82E08A95F1F700C0E3
:1093600026B199B18CB151BB479A422F46954370B3
:10937000E0E82E9F90011124422B292F2071422BCF
:10938000292F269526952870422B96959076492B65
:1093900090E0880F991F84709927482BA7EEA7B9F2
:1093A000F7EFFAB9E2EEEDB985E08A95F1F7000042
:1093B00047FF54C040FF52C051BB469A77B96AB9C3
:1093C0007DB915B8D8B96BB980E28EB9B1BB82E06E
:1093D0008A95F1F700C026B199B18CB151BB479A7B
:1093E000622F6695637050E8259F90011124622BCF
:1093F000292F2071622B292F269526952870622B04
:1094000096959076692B90E0880F991F8470992724
:10941000682BA7B9FAB9EDB985E08A95F1F7000094
:1094200044FD1AC08BE69AE10E947924CFBFFF91D8
:10943000EF91DF91CF91BF91AF919F918F917F91EC
:109440006F915F914F913F912F910F900BBE0F90B5
:109450000FBE0F901F9018950E948629CFBFE7CFAF
:109460001F920F920FB60F9211240BB60F922F93EB
:109470003F934F935F936F937F938F939F93AF939C
:10948000BF93CF93DF93EF93FF93CEE6D0E0888135
:109490008D7F888385B3876085BB78940E94460260
:1094A000F894888182608883FF91EF91DF91CF915A
:1094B000BF91AF919F918F917F916F915F914F91EC
:1094C0003F912F910F900BBE0F900FBE0F901F90EA
:1094D0001895CF93DF93CDB7DEB760970FB6F894AA
:1094E000DEBF0FBECDBF20E8209361001092610067
:1094F000F89414B817B81AB81DB810BA15B880EE99
:1095000088B91BB81EB893EE91BB0FEF04B987B9A9
:1095100037E03AB98DB990BB9CE797BD94B592609E
:1095200094BD95B5936095BD90916E0092609093B7
:109530006E00EC9A96EC91BB469A87B93AB98DB910
:1095400015B828B91BB81EB887E481BB32E03A953C
:10955000F1F700C086B189B18CB191BB479A87EE13
:1095600087B987EF8AB982EE8DB987EB92E0E6E49E
:10957000F0E1DF01AC011D9241505040E1F7EBEC0E
:10958000F9E0DF011D922A95E9F781E4EBE4FAE0C6
:10959000DF011D928A95E9F710E210935A0A85E4DB
:1095A000EDEFFFE0DF011D928A95E9F786E6E7E936
:1095B000FFE0DF011D928A95E9F70093FC0F0E94FE
:1095C000AE1782E691E0ECE8FAE0DF019C011D9223
:1095D00021503040E1F78FE38093EB0B46E050E001
:1095E0006FEF70E084EE9BE00E94CA551092E40B8E
:1095F0000E94862983E191E0EEEEFBE0DF019C0111
:109600001D9221503040E1F740E850E06FEF70E0EC
:109610008FEE9BE00E94CA5540E850E06FEF70E08B
:1096200087E79CE00E94CA5587E8E1E0FDE0DF01A2
:109630001D928A95E9F740E850E06FEF70E0CF01A6
:109640000E94CA558FEF9FEF9093820D8093810DFA
:109650000093830D85E1E1E7F3E1DF011D928A9537
:10966000E9F700937213009374138FEF9FEFDC01FF
:109670008093751390937613A0937713B093781318
:1096800081E08093731300937F13009383131092F0
:10969000A8191092AA191092A91980EC80936D1A3A
:1096A0008BEA99E190936F1A80936E1A10926C1A5C
:1096B00010926B1A10928C1910928B1910929019AB
:1096C00010928F1910929419109293191092961962
:1096D00010929519109298191092971910929C193E
:1096E00010929B191092A01910929F191092A21912
:1096F0001092A1191092A4191092A31983E49DE36A
:10970000909384198093831985EC9BE39093881937
:109710008093871982EB9BE390938A198093891930
:1097200088EE92E290938619809385198DE092E2FB
:1097300090939219809391198DED9EE190938E19DB
:1097400080938D198BE399E490939E1980939D19D2
:109750008EEB93E290939A198093991910928E0D43
:1097600010928D0D10938A0D83EB94E190938C0DE4
:1097700080938B0D1092890D1092880D80E090E0FF
:109780006AE2689F9001699F300D1124A9014E5B28
:109790005E4EDA01462F1D924A95E9F72A5B3F4E4D
:1097A000D901262F1D922A95E9F701968630910559
:1097B00041F78EE392E10E946E1989E592E10E94E1
:1097C0006E1981E0809373128091591290915A1210
:1097D000A0915B12B0915C12892B8A2B8B2B51F4D8
:1097E00060918F0D7091900D8091910D9091920DDF
:1097F0000E9431560E942E566093591270935A124D
:1098000080935B1290935C1280917112843011F1FD
:1098100084E08093711289E592E10E944414A09142
:109820007212BB27A1950CF4B095AA0FBB1F11961D
:109830002091611230916212409163125091641232
:109840000E9473566093651270936612809367123C
:109850009093681286EC81BB469A90EE97B927E008
:109860002AB99DB991E095B990E498B91BB890E2F6
:109870009EB997E491BB32E03A95F1F700C096B1FA
:1098800099B12CB181BB479A87EE87B987EF8AB926
:1098900082EE8DB994FD6DC28BED90E00E94DD16D5
:1098A000811106C00E9496158BED90E00E94CF4377
:1098B0001FB7F89462E08CED90E00E9415168823A3
:1098C00009F455C28FE38093AD141092AF14109237
:1098D000B01480E090E89093B2148093B11460913A
:1098E000960F662309F499C08091940F9091950F7B
:1098F000FC0120E030E074E2729FD001739FB00D54
:109900001124AA57BC4E6F0144E2C40ED11C4191F0
:1099100051914D935D93EC15FD05C9F72F5F3F4FB6
:109920002830310549F7FC01E05EFE4F208131818E
:109930003093A9142093A814FC01EE5DFE4F208102
:109940003181FC01EC5DFE4FF093950FE093940F95
:109950003093A7142093A6142081FC01EB5DFE4FE9
:10996000F093950FE093940F2093AA142081FC01AB
:10997000EA5DFE4FF093950FE093940F2093AB14A4
:10998000623008F44AC02081FC01E95DFE4FF0938B
:10999000950FE093940F2093AD142081FC01E85DB6
:1099A000FE4FF093950FE093940F2093AC14623028
:1099B000A1F12081FC01E75DFE4FF093950FE0934C
:1099C000940F2093AE14633041F12081FC01E65DD9
:1099D000FE4FF093950FE093940F2093AF146430F3
:1099E000E1F02081FC01E55DFE4FF093950FE093DF
:1099F000940F2093B014653081F020813181835D14
:109A00009E4F9093950F8093940F3093B2142093B0
:109A1000B114663011F01FBF25C081E01FBF811156
:109A200021C01FB7F8948DE291E0E6E8F3E1DF0191
:109A30009C011D9221503040E1F780E090E8909326
:109A4000A7148093A6142FEF2093AB142FE3209339
:109A5000AD149093B2148093B1140E94AE171FBF3F
:109A60000E943B1A81E00E94242A00E210E076E185
:109A7000D72E8091FB0F0E94D70E8091FB0F803173
:109A800009F472C1992787FD909501968F7190789E
:109A900097FF04C00197806E9F6F01968093FB0F24
:109AA0000150110931F764E1C62E66E0D62E00E1BF
:109AB00016E0D8018D918D010E94D70EB6E00431D9
:109AC0001B07B9F700910E0110910F01A090120130
:109AD000B0901301809010019090110198012A1903
:109AE0003B092819390940E050E0412C512C612CE8
:109AF00080E8782EC301B2010E94B456209314016D
:109B0000309315014093160150931701940120954D
:109B100030952A193B09201B310B40E050E0C3016E
:109B2000B2010E94B456209318013093190140935A
:109B30001A0150931B010091A6141091A7141093C1
:109B40000101009300018090040190900501A09014
:109B50000201B09003019801281939092A193B091B
:109B600040E050E0C301B2010E94B45620930601C8
:109B70003093070140930801509309019501209506
:109B8000309528193909201B310B40E050E0C30102
:109B9000B2010E94B45620930A0130930B01409306
:109BA0000C0150930D010E94B2220E94A8216FEF78
:109BB0008FEF0E94C6258EE697E00E94821378946C
:109BC00096EC692EAA24A39422E4722E30E5832E0B
:109BD00047E8942E56E1B52E9FB7F8948091D314A0
:109BE0008F5F8093D31461BA469A80FBEE24E0F82D
:109BF000F12CEE0CFF1CEE0CFF1CE1E3EE2A8E2D87
:109C000086958270806CA5B878B88BB88EB991BAF9
:109C10009FBF1092970F1092980F1092990F109269
:109C20009A0FFFEFF093FC0F04E010E00DC09927AE
:109C300087FD909501968F71907897FD01C2809372
:109C4000FB0F0150110969F08091FB0F0E94D70EA4
:109C50008091FB0F803159F7B092FB0F0150110931
:109C600099F700E116E0D8018D918D010E94D70E81
:109C7000C016D106C1F78091FC0F8F3F11F480917F
:109C8000741380937413873109F4DFC181E09091DC
:109C9000AA14911180E00E947840609174136F3F84
:109CA00009F44FC0E62FEE0FFF0BE554F04F008193
:109CB00011811801412C512C8091751390917613CC
:109CC000A0917713B0917813281639064A065B06DF
:109CD000C1F120927513309276134092771350920F
:109CE000781310937A1300937913862F0E949D178F
:109CF0008823C9F0A0910E01B0910F01E0911201EB
:109D0000F09113016091100170911101CB018095C8
:109D100090958017910708F0C1C28FEF9FEF909345
:109D20007A13809379130E948A318091741386315B
:109D300009F4D3C2803109F4DBC28450883008F4BE
:109D4000AAC28091D3148370823009F41AC283307E
:109D500009F4CFC1813009F4B8C10E941D1C6FEF16
:109D600080E00E94C62538CFD092FB0F99CE80E0CC
:109D700055CE0E94F93D712CA12CB12C46EC542EED
:109D80004424439450E4652E67E8262E70EE372E67
:109D90000FEF1FEF5FB7F89451BA469A45B868B80D
:109DA0001BB81EB821BA4DE04A95F1F7000051BA30
:109DB000469A37B867E06AB93DB845B868B81BB885
:109DC0006EB887E481BB92E09A95F1F700C026B1A6
:109DD00099B18CB151BA479A422F46954370A0E889
:109DE0002A9F90011124422B292F2071422B292FC9
:109DF000269526952870422B96959076492B90E0D3
:109E0000880F991F84709927482BB7EEB7B9E7EFF1
:109E1000EAB9F2EEFDB95FBF41FF09C1C501019684
:109E200062E170E0B5D2782EA82EB12C7092930D1D
:109E30002BE0271508F0F8C08FEF9FEF90933E10AE
:109E400080933D109BEA799E912D112496959695CD
:109E5000892F880F890F880F472D481B50E0A5E2F6
:109E6000B0E1E1E0F0E180E090E00EC020E030E021
:109E70002D933D93118F008F0193119313870287C8
:109E800001968630910531F08417950779F72FEF09
:109E90003FEFEECF35E0371508F4BCC08FEF9FEFF2
:109EA000909334108093331080914110816080939F
:109EB00041100E940C11872D8650863008F087C013
:109EC000AFEFBFEFB0933610A093351080914110E3
:109ED0008860809341100E940C114501880C991CE8
:109EE00041E050E1840E951E83E99BE5D4018D93FA
:109EF0009C9388E00E94813E6B017C0182EA9BEB8F
:109F0000F4019183808380E80E94813EAB01BC0113
:109F100010922610109225101092281010922710DF
:109F200010922A101092291010922C1010922B10BF
:109F300010922E1010922D101092301010922F109F
:109F40004C195D096E097F09C52ED62EE72EFF2418
:109F5000E7FCFA94F4E6CF16D104E104F1042CF006
:109F6000B3E6CB2ED12CE12CF12C2DE9C2162FEF2C
:109F7000D206E206F20634F4ADE9CA2EDD24DA9404
:109F8000ED2CFD2CB601D7FC57C0882777FD8095B6
:109F9000982F0E94ED19C701B601662797FD6395BA
:109FA00077278827992740E089E00E94BE19F2E3CD
:109FB000FF2E8FE39CE90197F1F700C0000081E0DC
:109FC0000E94FF0F0E946C3DFA9499F7E3CE109225
:109FD00036101092351080914110877F8093411088
:109FE0000E940C119BE0971508F077CF4501880C73
:109FF000991C21E030E1820E931E83E094E6D401A7
:10A000008D939C9388E00E94813E6B017C0186ECDD
:10A0100094E976CF10923410109233108091411051
:10A020008E7F8093411045CF80E090E007CF42FFC4
:10A03000FDCEC5014196F4CE719561957109A5CF0C
:10A040000197806E9F6F0196FACD60917F1367FD37
:10A050001DCE4090E90F5090EA0F920140E050E091
:10A060008091751390917613A0917713B091781326
:10A07000281739074A075B0709F408CE772767FDD9
:10A080007095CB01880F991F860F971F880F991F16
:10A09000880F991F805E9A4FFC01DE0111966CE0DB
:10A0A00001900D926A95E1F7FC0110810181111177
:10A0B00098C0E02FEE0FFF0BE95EFC4E518240820C
:10A0C000A09273130E94A821E1CD60913D1370917D
:10A0D0003E1388E10E94C7296091271370912813CD
:10A0E0008EE10E94C72960E070E68DE10E94C729D9
:10A0F00036CE0E94643400E010E423E035E440E012
:10A1000050EE6BE276E480914313909144130E94E9
:10A11000C1139C019093F3128093F21281E0203DD1
:10A1200037400CF080E08093F412809151139091AD
:10A130005213811554E0950708F4A6C02091AE147F
:10A14000222309F4E4C0A0E0B0E0880F991FAA1F01
:10A15000BB1F880F991FAA1FBB1F880F991FAA1F1B
:10A16000BB1F880F991FAA1FBB1FFD01EE0FFF1F0A
:10A17000EC5EF94F8081918190934510809344105B
:10A18000EECD6091191370911A1389E10E94C729CD
:10A1900060911F13709120138AE10E94C72980915A
:10A1A000D70F9091D80F4091F0125091F11266277D
:10A1B00057FD6095762F480F591F611D711D77FD62
:10A1C00088C0CB01BA016115710531E083079105A3
:10A1D00024F06FEF7FEF80E090E08BE10E94C729D1
:10A1E000BECD133008F06CCF4D863E874F87588B1D
:10A1F0000E94A813FE01359660E070E0CB012D852A
:10A200003E854F855889A191B191AB2B49F06F5F85
:10A210007F4F8F4F9F4F643071058105910599F7EE
:10A22000A8D01C01552437FC5094452C80917B13F9
:10A2300090917C13A0917D13B0917E13281639065E
:10A240004A065B0671F0F1013296EE0FFF1F21E026
:10A2500030E02C0F3D1FE20FF31F808191810E949F
:10A260008213113009F04DC0E02FFF27E7FDF09574
:10A27000E350FD4E208220927B1330927C1340925B
:10A280007D1350927E131CCF8FEF9FEF909345105C
:10A290008093441064CD0E942F2053CD06171707DA
:10A2A00008F444C0CD018E1B9F0B0817190708F056
:10A2B00040C0A2019101261B370B41095109609151
:10A2C000140170911501809116019091170151D0E0
:10A2D00026CD40E050E0BA0174CF6091E70F709155
:10A2E000E80F21E042E080E090E00E94941D29CD3B
:10A2F0000E94223121E041E060E070E00E94941D64
:10A3000020CDB201A101802F0E94961FB4CF00E0A2
:10A3100010E02AEF33E440E050EE6BEA76E40E946E
:10A32000C113909345108093441019CD80E090E0C4
:10A33000F6CCCF018A0F9B1F8017910718F080E0A1
:10A3400090E8EDCCA2019101281B390B410951097C
:10A35000609118017091190180911A0190911B016F
:10A3600008D09058DCCCF4D4B7FF0895821B930B2F
:10A370000895DB018F939F93ACD4BF91AF91A29FBF
:10A38000800D911DA39F900DB29F900D11240895F3
:10A3900097FB072E16F4009406D077FD08D0A9D4B9
:10A3A00007FC05D03EF4909581959F4F08957095D8
:10A3B00061957F4F08955058BB27AA270ED0F1C151
:10A3C000BAD130F0BFD120F031F49F3F11F41EF428
:10A3D0008AC10EF4E095E7FB80C1E92F04D280F337
:10A3E000BA17620773078407950718F071F49EF592
:10A3F0001CC20EF4E0950B2EBA2FA02D0B01B90153
:10A4000090010C01CA01A0011124FF27591B99F0EA
:10A41000593F50F4503E68F11A16F040A22F232FF6
:10A42000342F4427585FF3CF469537952795A79546
:10A43000F0405395C9F77EF41F16BA0B620B730BED
:10A44000840BBAF09150A1F0FF0FBB1F661F771F5E
:10A45000881FC2F70EC0BA0F621F731F841F48F413
:10A46000879577956795B795F7959E3F08F0B3CF99
:10A470009395880F08F09927EE0F97958795089583
:10A4800008D108F481E0089565D1E3959BC10CD013
:10A4900088C158D140F04FD130F021F45F3F19F01E
:10A4A0001CC15111C3C11FC19ED198F39923C9F397
:10A4B0005523B1F3951B550BBB27AA2762177307CA
:10A4C000840738F09F5F5F4F220F331F441FAA1F7E
:10A4D000A9F333D00E2E3AF0E0E830D0915050403E
:10A4E000E695001CCAF729D0FE2F27D0660F771FEC
:10A4F000881FBB1F261737074807AB07B0E809F0CE
:10A50000BB0B802DBF01FF2793585F4F2AF09E3F62
:10A51000510568F0E2C08AC15F3FECF3983EDCF37E
:10A52000869577956795B795F7959F5FC9F7880FDB
:10A53000911D9695879597F90895E1E0660F771F2D
:10A54000881FBB1F621773078407BA0720F0621BBE
:10A55000730B840BBA0BEE1F88F7E095089519F47E
:10A560000EF0BBC062C1BFC046D1C8F39638C0F779
:10A5700007F80F92E8942BE33AEA48EB5FE7DED165
:10A580000F920F920F924DB75EB70F9296D1ECEAF1
:10A59000F0E0ACD04F915F91EF91FF91E595EE1F08
:10A5A000FF1F49F0FE57E0684427EE0F441FFA955D
:10A5B000E1F74195550B4DD10F9007FE41C108952C
:10A5C0001AD188F09F5790F0B92F9927B751A0F072
:10A5D000D1F0660F771F881F991F1AF0BA95C9F737
:10A5E00012C0B13081F021D1B1E008951EC1672FB2
:10A5F000782F8827B85F39F0B93FCCF386957795E7
:10A600006795B395D9F73EF49095809570956195CF
:10A610007F4F8F4F9F4F0895E89409C097FB3EF4FA
:10A6200090958095709561957F4F8F4F9F4F99239F
:10A63000A9F0F92F96E9BB279395F695879577951D
:10A640006795B795F111F8CFFAF4BB0F11F460FFDD
:10A650001BC06F5F7F4F8F4F9F4F16C0882311F035
:10A6600096E911C0772321F09EE8872F762F05C049
:10A67000662371F096E8862F70E060E02AF09A95E4
:10A68000660F771F881FDAF7880F9695879597F9D9
:10A690000895990F0008550FAA0BE0E8FEEF161673
:10A6A0001706E807F907C0F012161306E407F507C6
:10A6B00098F0621B730B840B950B39F40A2661F03A
:10A6C000232B242B252B21F408950A2609F4A140DD
:10A6D000A6958FEF811D811D089597F99F6780E8EA
:10A6E00070E060E008959FEF80EC0895DF93CF93D2
:10A6F0001F930F93FF92EF92DF927B018C0168947E
:10A7000005C0DA2EEF0118D1FE01E894A59125913C
:10A71000359145915591AEF3EF015FDEFE01970152
:10A72000A801DA9479F7DF90EF90FF900F911F91D5
:10A73000CF91DF91089500240A9416161706180683
:10A740000906089500240A94121613061406050635
:10A750000895C9CF50D0E8F3E894E0E0BB279F57B5
:10A76000F0F02AED3FE049EC06C0EE0FBB0F661F8C
:10A77000771F881F28F0B23A62077307840728F012
:10A78000B25A620B730B840BE3959A9572F780387B
:10A7900030F49A95BB0F661F771F881FD2F7904839
:10A7A00070C1092E0394000C11F4882352F0BB0FE2
:10A7B00040F4BF2B11F460FF04C06F5F7F4F8F4FD9
:10A7C0009F4F0895EF93E0FF06C0A2EA2AED3FE015
:10A7D00049EC5FEB02DEE5DF0F90039401FC90583B
:10A7E000E4EDF0E05AC157FD9058440F551F59F061
:10A7F0005F3F71F04795880F97FB991F61F09F3F6E
:10A8000079F087950895121613061406551FF2CF96
:10A810004695F1DF08C0161617061806991FF1CFE6
:10A8200086957105610508940895E894BB2766270D
:10A830007727CB0197F908952CDF08F48FEF08955F
:10A840009B01AC0160E070E080E89FE320CE45CF43
:10A8500016C1D1DFE8F39923D9F3940F511DBBF34F
:10A860009150504094F059F0882332F0660F771FD2
:10A87000881F91505040C1F79E3F510544F7880F03
:10A88000911D9695879597F908955F3FACF0983E96
:10A890009CF0BB27869577956795B79508F4B160CE
:10A8A0009395C1F7BB0F58F711F460FFE8CF6F5FC6
:10A8B0007F4F8F4F9F4FE3CFB9CFFA01DC01AA0F33
:10A8C000BB1F9B01AC01BF5728F422273327442725
:10A8D00050781FC0B75188F4AB2F002446953795A8
:10A8E0002795011CA395D2F3002069F0220F331F96
:10A8F000441FB395DAF30DD05ECD61307105A0E849
:10A900008A07B94630F49B01AC0166277727882770
:10A910009078309621F020833183428353830895C9
:10A920000BD03FCF08DF28F00DDF18F0952309F09A
:10A93000D4CED9CE11247ACF56DFA0F3959FD1F390
:10A94000950F50E0551F629FF001729FBB27F00DDD
:10A95000B11D639FAA27F00DB11DAA1F649F662732
:10A96000B00DA11D661F829F2227B00DA11D621F81
:10A97000739FB00DA11D621F839FA00D611D221F3B
:10A98000749F3327A00D611D231F849F600D211D1F
:10A99000822F762F6A2F11249F5750408AF0E1F0C2
:10A9A00088234AF0EE0FFF1FBB1F661F771F881F0B
:10A9B00091505040A9F79E3F510570F08ECE36CF92
:10A9C0005F3FECF3983EDCF3869577956795B795F6
:10A9D000F795E7959F5FC1F7FE2B880F911D969520
:10A9E000879597F90895FA01EE0FFF1F309621051C
:10A9F000310599F16115710561F48038BFE39B075A
:10AA000049F168949038810561F08038BFEF9B0769
:10AA100041F0992342F5FF3FE1053105210511F190
:10AA2000E8940894E795D901AA2329F4AB2FBE2F07
:10AA3000F85FD0F310C0FF5F70F4A695E0F7F73928
:10AA400050F019F0FF3A38F49F779F930CD00F9095
:10AA500007FC905808953EF046CE60E070E080E834
:10AA60009FE308954FE79F775F934F933F932F9313
:10AA70002AD02F913F914F915F9152DF75CD9F3F2B
:10AA800031F0915020F4879577956795B795880FA9
:10AA9000911D9695879597F908959F938F937F932E
:10AAA0006F93FF93EF939B01AC013ADFEF91FF911E
:10AAB0001DDE2F913F914F915F9132CF0EF0DFCF8E
:10AAC00012CE68940ACE97DEC8F39923D1F3C6F369
:10AAD000DF93CF931F930F93FF92C92FDD27882316
:10AAE0002AF02197660F771F881FDAF720E030E001
:10AAF00040E85FEB9FE3883920F0803E30F02196FC
:10AB00008F775ADCE2EFF0E003C056DCEFE1F1E0D2
:10AB1000EDDD8B01BE01EC01FB2E6F5771097595C0
:10AB2000771F880B990B7ADD28E132E741E35FE379
:10AB300003DFAF2D9801AE01FF900F911F91CF91D0
:10AB4000DF914BDC2ECEFB01DC0104C08D91019026
:10AB5000801921F441505040C8F7881B990B089583
:10AB6000FB01DC0102C001900D9241505040D8F72A
:10AB700008956817790768F4FB01DC01E40FF51FFD
:10AB8000A40FB51F02C002900E9241505040D8F75A
:10AB90000895E6CFDC0101C06D9341505040E0F7CD
:10ABA0000895FB01DC010D900020E9F71197019059
:10ABB0000D920020E1F70895FB01DC0101900D9258
:10ABC0000020E1F708958F929F92AF92BF92CF92AB
:10ABD000DF92EF92FF92CF93DF93EC01688179814E
:10ABE0008A819B81611571058105910521F464E2DB
:10ABF00079ED8BE597E02DE133EF41E050E08DD02A
:10AC000049015A019B01AC01A7EAB1E462D06B0192
:10AC10007C01ACEEB4EFA501940167D0C60ED71E3F
:10AC2000E81EF91EF7FE06C081E0C81AD108E10847
:10AC300080E8F80AC882D982EA82FB82E894F7F8B1
:10AC4000B601C701DF91CF91FF90EF90DF90CF90D9
:10AC5000BF90AF909F908F900895B5CF8CE191E019
:10AC6000B2CF60931C0170931D0180931E019093DD
:10AC70001F010895FB019F01E8944230BCF045326A
:10AC8000ACF44A3029F497FB1EF4909581959F4FC0
:10AC9000642F77272ED0805D8A330CF0895D8193F5
:10ACA000CB010097A9F716F45DE251931082C90118
:10ACB00000C0DC01FC01672F71917723E1F7329727
:10ACC00004C07C916D9370836291AE17BF07C8F387
:10ACD00008953ED0A59F900DB49F900DA49F800D28
:10ACE000911D11240895B7FFF4CFF3DF821B930B5E
:10ACF0000895AA1BBB1B51E107C0AA1FBB1FA617C3
:10AD0000B70710F0A61BB70B881F991F5A95A9F714
:10AD100080959095BC01CD010895052E97FB16F402
:10AD2000009406D057FD0CD01FD007FC09D07EF44C
:10AD300090958095709561957F4F8F4F9F4F0895A7
:10AD400050954095309521953F4F4F4F5F4F089557
:10AD5000A29FB001B39FC001A39F01D0B29F700D0D
:10AD6000811D1124911D0895A1E21A2EAA1BBB1B5F
:10AD7000FD010DC0AA1FBB1FEE1FFF1FA217B307C7
:10AD8000E407F50720F0A21BB30BE40BF50B661FDD
:10AD9000771F881F991F1A9469F7609570958095A1
:10ADA00090959B01AC01BD01CF010895F894FFCFB0
:10ADB00000809001000C00000000000000000080F6
:10ADC000000000080000000000000000010000007A
:10ADD00000006207640E3415D21B41228128942E94
:10ADE0007B34383ACB3F37457B4A994F9254675969
:10ADF0001A5EAB621A676A6B9B6FAD73A2777B7B3F
:10AE0000387FD9826186CF89258D62908893989604
:10AE10009199759C449FFFA1A6A43AA7BBA92AAC0F
:10AE200088AED5B011B33DB559B766B964BB54BD52
:10AE300036BF0BC1D2C28CC43AC6DCC772C9FDCAC8
:10AE40007CCCF1CD5BCFBBD011D25ED3A1D4DBD50E
:10AE50000CD734D854D96DDA7DDB85DC86DD80DE15
:10AE600073DF5FE044E123E2FCE2CEE39BE461E5D3
:10AE700022E6DEE695E746E8F2E89AE93DEADBEA13
:10AE800074EB0AEC9BEC28EDB1ED36EEB8EE36EF44
:10AE9000B0EF27F09AF00BF178F1E2F149F2ADF260
:10AEA0000EF36DF3C9F322F479F4CDF41FF56FF5C9
:10AEB000BCF507F651F698F6DDF620F761F7A0F736
:10AEC000DEF71AF854F88DF8C4F8F9F82DF95FF99F
:10AED00090F9C0F9EEF91BFA47FA71FA9BFAC3FA36
:10AEE000EAFA10FB35FB58FB7BFB9DFBBEFBDEFB50
:10AEF000FDFB1BFC38FC55FC70FC8BFCA5FCBFFC6F
:10AF0000D8FCF0FC07FD1EFD34FD49FD5EFD72FD21
:10AF100086FD99FDABFDBDFDCFFDE0FDF0FD01FE21
:10AF200010FE1FFE2EFE3CFE4AFE58FE65FE72FE1F
:10AF30007EFE8AFE96FEA2FEADFEB7FEC2FECCFEEF
:10AF4000D6FEE0FEE9FEF2FEFBFE04FF0CFF14FF5E
:10AF50001CFF23FF2BFF32FF39FF40FF47FF4DFF50
:10AF600053FF59FF5FFF65FF6BFF70FF75FF7BFFAE
:10AF700080FF84FF89FF8EFF92FF96FF9BFF9FFF5C
:10AF8000A3FFA7FFAAFFAEFFB1FFB5FFB8FFBBFF4E
:10AF9000BFFFC2FFC5FFC8FFCAFFCDFFD0FFD2FF72
:10AFA000D5FFD7FFDAFFDCFFDEFFE0FFE3FFE5FFC1
:10AFB000E7FFE9FFEAFFECFFEEFFF0FFF1FFF3FF31
:10AFC000F5FFF6FFF8FFF9FFFBFFFCFFFDFFFFFFBA
:10AFD0000000EE01DA03C305A9078C096C0B4A0DCA
:10AFE000250FFD10D212A414741641180B1AD31B8E
:10AFF000981D5A1F1A21D72291244926FE27B129CC
:10B00000612B0E2DB92E62300832AB334D35EB3645
:10B010008738213AB93B4E3DE03E7140FE418A43BC
:10B0200013459A461F48A149224B9F4C1B4E944FF3
:10B030000C518152F4536455D3563F58A959115BB2
:10B04000775CDB5D3D5F9C60FA615663AF640766C9
:10B050005C67B068016A516B9E6CEA6D346F7B70FF
:10B06000C171057347748775C57602783C79757A26
:10B07000AC7BE17C147E457F7580A381CF82F98310
:10B08000218548866D879188B289D28AF18B0D8D92
:10B09000288E418F59906F9183929693A794B6957D
:10B0A000C496D197DB98E599EC9AF29BF79CFA9DB0
:10B0B000FB9EFB9FFAA0F7A1F2A2ECA3E5A4DCA5FE
:10B0C000D2A6C6A7B9A8AAA99AAA88AB76AC61AD40
:10B0D0004CAE35AF1CB003B1E7B1CBB2ADB38EB45B
:10B0E0006EB54CB629B705B8DFB8B8B990BA67BB2A
:10B0F0003CBC10BDE3BDB4BE85BF54C022C1EEC18F
:10B10000BAC284C34DC415C5DCC5A2C666C729C86A
:10B11000ECC8ADC96DCA2BCBE9CBA5CC61CD1BCE9C
:10B12000D4CE8DCF44D0FAD0AFD162D215D3C7D30D
:10B1300078D427D5D6D584D630D7DCD786D830D9A1
:10B14000D9D980DA27DBCCDB71DC15DDB7DD59DE40
:10B15000FADE9ADF39E0D7E074E110E2ACE246E3D0
:10B16000DFE378E410E5A6E53CE6D1E665E7F9E73C
:10B170008BE81CE9ADE93DEACCEA5AEBE7EB74EC6D
:10B1800000ED8AED14EE9EEE26EFAEEF35F0BBF04B
:10B1900040F1C4F148F2CBF24DF3CEF34FF4CFF4CB
:10B1A0004EF5CCF54AF6C7F643F7BEF739F8B3F8D3
:10B1B0002CF9A5F91DFA94FA0AFB80FBF5FB6AFC51
:10B1C000DDFC50FDC3FD34FEA5FE16FF85FFF4FF38
:10B1D000001D9607000000000000000002009C0710
:10B1E000A407AD07B5070000001ABE070000000065
:10B1F00000000000001BC607000000000000000067
:10B200000019CE0700000000000000000202D6076F
:10B21000DE07E707F007F80701140008100909081E
:10B220000D081108001615080000000000000000BD
:10B23000001C1B080000000000000000001722088E
:10B240000000000000000000001D96070000000044
:10B250000000000002012A0832083A0833083508C5
:10B26000010A3C08440848080000000002054D0897
:10B27000550844084808590801175E0866086A0816
:10B280000000000002036E08DE07E707F007F8077A
:10B29000020476087F08830887088B0801128F084C
:10B2A0009408440848080000011699089F08A4085B
:10B2B000A90800000018AD08000000000000000010
:10B2C00001101E1DC000A800900080006000480012
:10B2D00030002400180012000C00090006000400D1
:10B2E00003000200080C080A0808080808080808F3
:10B2F000080A080C0C0000000000080C0A0A0A0AE0
:10B300000A0C0C0800000000000000000000000013
:10B31000000000000000000000000000000000002D
:10B3200000000000003022366D247D20390F764663
:10B33000104010523F065B4F666D7D077F6F484897
:10B34000614843277B777F393F79713D76060E76DA
:10B350003837373F733F776D783E3E7E76665B3990
:10B36000640F230802777C585E79716F74040C7443
:10B370003837545C7367506D781C1C7E766E5B3971
:10B38000300F010001010101010101010103020669
:10B3900002010101000102040203020102017472B0
:10B3A000616E7370203D20000000000000007D09E8
:10B3B000820986098A098E09920996099A099E09C5
:10B3C000A209A609AB09B009B509BA09BF09C409A0
:10B3D000FCFDFE010204081020408000FFFFFFFF7B
:10B3E000FF1E00181D0C0D1F0102030405060708AF
:10B3F000090A0B191B1A1CFFFFFFFFFFFFFFFF02CB
:10B4000003020000010001010101010001010037F8
:10B4100056656F7C878B8F949AA4B0B9BFD2476C66
:10B4200069476C6927732050363030207570677219
:10B4300061646520616C706861204D617920203203
:10B440002032303135007370656564006C666F20A2
:10B450007368700070756C732D74726900726E641D
:10B460002D73696E006E6F69732D73617700566975
:10B4700062207370640056696220616D74006D6FA4
:10B480006420646C7900616D70207368700066617F
:10B4900073742D65787000666173742D6C696E002D
:10B4A000736C6F2D65787000736C6F2D6C696E0016
:10B4B00062656E64207467740056636F005663663D
:10B4C00000566F6C00676C69646500646574756E26
:10B4D0006500616D702056656C006C666F20746746
:10B4E000740061620061622D566361006C666F20BA
:10B4F00072616E006C6F770068696768006D6F64D9
:10B500002072616E006D696E0066756C6C006D6F07
:10B510006420746774006C666F0056696200666927
:10B520006C207368700062656E642072616E003218
:10B530006E640033726400357468004F6374007089
:10B5400072696F006C61737400706974636800667F
:10B550007265650073656D69006F63740066696C80
:10B560002056656C0062656E6465722063616C696B
:10B5700062726174656400707265736574732064CF
:10B58000756D706564002072656376002073656E6A
:10B590006400707265737320616761696E20666F05
:10B5A000722062656E6465722063616C69627261AB
:10B5B00074696F6E0056632D206F6E0056632D20E8
:10B5C0006F666600707265737320616761696E20D3
:10B5D000746F2064756D702070726573657473008C
:10B5E000496E742073796E63004D696469207379C4
:10B5F0006E6300746170652073796E63007370729E
:10B600006561642000202F20566366206C696D20E0
:10B6100000707265737320616761696E20666F7276
:10B62000206261736963207061746368006F6D6E7E
:10B6300069006368310063683200636833006368DF
:10B6400034006368350063683600636837006368F8
:10B650003800636839006368313000636831310055
:10B6600063683132006368313300636831340063EA
:0AB6700068313500636831360000D0
:020000021000EC
:10E000002F923F924F925F926F927F928F929F9248
:10E01000AF92BF92CF92DF92EF92FF920F931F9336
:10E02000CF93DF93CDB7DEB728970FB6F894DEBF56
:10E030000FBECDBF2FEF31EE44E0215030404040C5
:10E04000E1F700C00000F89414B817B81AB81DB86A
:10E0500010BA15B890EE98B91BB81EB883EE81BB04
:10E060002FEF24B997B947E04AB99DB980BB36EC88
:10E0700031BB469A97B94AB99DB915B880E888B9B5
:10E080001BB81EB8F7E4F1BB62E06A95F1F700C077
:10E0900086B189B18CB131BB479AE7EEE7B977EF2A
:10E0A0007AB962EE6DB931BB469AA1E0A5B982E4B6
:10E0B00088B91BB81EB887E881BB8DE08A95F1F757
:10E0C000000031BB469A97B94AB99DB9A5B920E479
:10E0D00028B91BB82EB9F1BBB2E0BA95F1F700C070
:10E0E00086B159B1BCB131BB479AE7B97AB96DB9BC
:10E0F000BDE0BA95F1F7000031BB469A97B94AB92D
:10E100009DB9A5B928B91BB82EB9F1BBF2E0FA95B3
:10E11000F1F700C026B199B14CB131BB479AE7B9CC
:10E120007AB96DB93DE03A95F1F70000422F469576
:10E13000437060E8269F90011124242B392F307101
:10E14000322B292F269526952870232B969590768D
:10E15000922B907C21E0903C09F020E0382F3695FE
:10E160003370A0E88A9FC0011124832B952F9071F2
:10E17000982B852F869586958870982B852F869568
:10E180008076982B907C81E0903C09F080E082239F
:10E1900009F4EEC186EC81BB469A21E025B990E4F2
:10E1A00098B99BB91EB897E891BBBAE0BA95F1F758
:10E1B00000C081BB469A25B934E438B930E73BB991
:10E1C00032E23EB991BBEAE0EA95F1F700C081BBCB
:10E1D000469A25B922E428B920E52BB920EC2EB9BE
:10E1E00091BBFAE0FA95F1F700C081BB469A15B8E9
:10E1F00026E828B923E02BB91EB891BBAFE9BFE0F0
:10E200001197F1F700C0000081BB469A15B823E8CA
:10E2100028B923E12BB922E02EB991BBBAE0BA9517
:10E22000F1F700C081BB469A20EE27B997E09AB972
:10E230002DB915B870E878B99BB91EB867E461BB11
:10E24000E2E0EA95F1F700C036B139B13CB181BBEB
:10E25000479A57EE57B947EF4AB932EE3DB9F5E064
:10E26000FA95F1F7000081BB469A27B99AB92DB902
:10E2700015B878B99BB990E29EB961BB22E02A95A6
:10E28000F1F700C096B199B19CB181BB479A57B9DB
:10E290004AB93DB935E03A95F1F7000099249394D5
:10E2A0000F2EF6E82F2EF8E13F2EF02D0F2EF6E878
:10E2B0004F2EF9E15F2EF02D88248394BED499234C
:10E2C0000CF441C1803F9105C9F7B7D4892B09F0FF
:10E2D0003AC1B3D48136910509F035C1AED4469721
:10E2E00009F031C1AAD48B36910509F02CC1A5D40F
:10E2F0007C0199230CF427C1682F80E090E080D442
:10E300008C01E894E7F8FF24F694FE2CEE24F794B1
:10E31000E79493D46C0199230CF415C1682FC801BC
:10E320006FD48C01E894C7F8DD24EC28FD28E114B3
:10E3300041E0F40621F0EF2809F407C104C17DD4BF
:10E340006C0199230CF4FFC0682FC80159D48C01CB
:10E3500074D45C0199230CF4F6C0682FC80150D422
:10E3600098878F83810169D47C0199230CF483C041
:10E37000682F8F81988544D498878F83C7018F77C2
:10E3800099279A83898359D47C0199230CF473C00B
:10E39000682F8F81988534D498878F83D701AF7782
:10E3A000BB27BC83AB8349D47C0199230CF463C0A5
:10E3B000682F8F81988524D498878F83F701EF7712
:10E3C000FF27FE83ED8339D47C0199230CF453C0DD
:10E3D000682F8F81988514D498878F833701E894AC
:10E3E00067F877242AD47C0199230CF444C0682F61
:10E3F0008F81988505D498878F83F8013397C7015B
:10E400009695982F8827979587952981822B8083C9
:10E41000F8013297C7018270992700249695879555
:10E420000794969587950794982F802D3B81832B91
:10E430008083F8013197C70184709927880F991F4D
:10E4400082959295907F9827807F98274D81842B85
:10E450008083C7018870992782959295907F98272D
:10E46000807F98278629D8018C930C5F1F4F041555
:10E47000150509F078CFE1D399230CF464C08C0121
:10E48000102F0027110FD9D399230CF45CC08F777C
:10E490009927880F991F880F991F082B192BCDD307
:10E4A00099230CF450C083709927082B192BEF8106
:10E4B000F8850E171F0709F046C0BFD3873F9105A7
:10E4C00009F041C0990CFFE3F91508F4982C26ECEB
:10E4D00021BB469A892D880F392D3695282F267015
:10E4E0002064992D991F9927991F292B992D907197
:10E4F000482F440F4072942B807C982B832F82707E
:10E50000806285B828B99BB98EB937E831BB4AE03B
:10E510004A95F1F700C0B5016F777727C6018F776D
:10E5200099279695982F882797958795682B792B0B
:10E53000CB01A0E0B0E06627782F892F9A2F43E81F
:10E5400058E15ED5BBCE89E701C08DE696EC91BB64
:10E55000469A982F9071906E86958270806221E025
:10E5600025B922E428B99BB98EB987E881BBFFCFD2
:10E5700028960FB6F894DEBF0FBECDBFDF91CF91C6
:10E580001F910F91FF90EF90DF90CF90BF90AF90D1
:10E590009F908F907F906F905F904F903F902F90C3
:02E5A0000895DC
:10EC00009C013627032E0294802D8F708327632F5B
:10EC10006025660F607E8627602D6327607F66957E
:10EC2000032E000C661F3695369536953F713627B4
:10EC30003227282F822F932F089545E04A95F1F728
:10EC40000000349B04C000C000C03499FCCF86ECA7
:10EC500081BB469A20EE27B997E09AB92DB915B82D
:10EC600020E828B99BB91EB897E491BB52E05A95A9
:10EC7000F1F700C096B129B13CB181BB479A87EE4C
:10EC800087B987EF8AB982EE8DB985E08A95F1F769
:10EC90000000392F3695337040E8949FC00111244D
:10ECA000832B922F9071892B922F96959695987021
:10ECB000892B26952076282B217B213809F040C00E
:10ECC00026EC21BB469A90EE97B987E08AB99DB9A8
:10ECD00015B890E898B98BB980E28EB987E481BB0A
:10ECE00052E05A95F1F700C036B199B14CB121BB51
:10ECF000479A87EE87B987EF8AB982EE8DB985E0AA
:10ED00008A95F1F70000832F8695837050E8359F30
:10ED100090011124282B892F8071282B892F86950B
:10ED200086958870282B96959076292B50E0CA01FD
:10ED3000880F991F84709927822B282F30E002C0FA
:0AED40002FEF3FEF822F932F08956D
:10F000008F929F92AF92BF92CF92EF92FF92CF9347
:10F01000DF93EA01CFB6F894F999FECF23E0FB0124
:10F0200080935B002093570010D707B600FCFDCFFC
:10F03000DE01B3954B015C0121E04881F980E12CB0
:10F04000F701E40FF11DAF0122960A01F401A0922D
:10F050005B0020935700F9D61124F2E08F0E911C2B
:10F06000A11CB11CAC17BD0741F725E0FB01809343
:10F070005B0020935700E9D607B600FCFDCF81E185
:10F0800080935700E2D6CFBEDF91CF91FF90EF90F3
:0CF09000CF90BF90AF909F908F9008959C
:00000001FF
